:020000041100E9
:10300000002373B52B4D2C4C28006361022601F080
:1030100061FA4021FE2221742800284B009601F01D
:10302000ABFA002836D1217CFF222800244B0096E1
:1030300001F0A2FA00282DD1224BA2899A4226D172
:10304000E389214A93420DD1204B6361204B2268D2
:10305000002A03D1002B01D043CB43C4280001F048
:1030600077FA73BD1B4A934201D00023EFE71A4B56
:103070001A4A1B68934206D9C02304222800217CE7
:103080009B0001F0EFFA114B6361154BDFE7002362
:103090002374EAE7CC233821AC2228009B01217459
:1030A00001F0E0FA0028F2D10E4B63610E4BE38190
:1030B0000E4BCCE7D443FF1F7463FF1F8063FF1FD9
:1030C0008263FF1F5959000083050000014300116E
:1030D00058BA0011821500009863FF1F8713000083
:1030E00064BA0011B9430011AAAAFFFF4CBA00113B
:1030F000F7B5164B0192C318021D002000938823D8
:103100005B05D3181B685C1C1AD09CB2402C18D8E5
:103110008D781E0CAC466746CD782D023D43AE42FD
:1031200006D1019800280ED110000C70240A4C70B2
:1031300003249BB20733A343D218009B9A42DED3E9
:10314000FEBD4432F9E71000FAE7C046FC0F00006C
:10315000802213B503000324019189B25201073183
:103160009B18A14304305A1A88235B05C3181B68B7
:10317000591C03D190429241104016BD99B240298A
:1031800007D80B000733A343C0189042ECD30020AC
:10319000F3E74430F9E7134B134A1B68126810B584
:1031A000FA24934201D81A00F824104BE4021B6859
:1031B0009A4210D813000E4A12689A420ED3013375
:1031C00007D1F823DB029C4203D10A49054808F0E5
:1031D0003FFB200010BDFC24E402ECE7FE24E402E7
:1031E000F7E7C04600C0071100D0071100E0071143
:1031F00000F00711FFFFFF7FF0B59BB015000490B2
:103200000391402A00D9A0E006AB59801A80FFF74D
:10321000C2FF0400042816D9002206A9FFF768FFA0
:10322000052810D906AB1B88AB420CD1002D07D066
:10323000514B2A000499C01808F05AFA002802D10C
:1032400001201BB0F0BD06AB1D8020000699FFF7E2
:103250007FFF041E7BD1069B0793FFF79CFF802313
:103260005B01C618802307001B039E4201D3F8268A
:10327000F60288235B05F31801931B68013302D023
:10328000019808F005FA3D49019808F0E1FA3B1D64
:103290000293331D05938822029B52059B181B68DD
:1032A00008935A1C3CD044219AB20091402A04D879
:1032B0000320D11D814389B2009103991B0C8B42DD
:1032C00024D0402A22D80122300008A9FFF710FF9D
:1032D000021E1BD1380008A9FFF70AFF04000428CA
:1032E00031D9009A059B9B1880225201B218934253
:1032F00040D288235B05C118009A09A808F038F964
:103300001D4B009A09A9F01808F09AF9009A029B3F
:103310009446634402931A4B029AFB189A42BAD31A
:1033200088235B05FC1821680198013908F090FAA0
:10333000200008F0ADF9039A07AB5A8030000799D6
:10334000FFF706FF0400002C03D1002079E70428D2
:10335000FBD988235B05E018069908F079FA032366
:10336000EA1C9A4300D16BE7034B0499E01808F07C
:1033700067F965E70424ECE704000011FFFFFF7F15
:10338000F80F0000F7B505001400402A21D80027E7
:1033900001AE71803780FFF7FEFE042816D93A008F
:1033A0003100FFF7A5FE042810D93688BC420BD0A7
:1033B000BD4209D0221CB44200D9321C064B92B245
:1033C000C118280008F0D4F830B2FEBDC04300B2E6
:1033D000FBE703204042F8E70400001137B5042260
:1033E00004000D0001A81649FFF7CCFF02000428D5
:1033F0000BD1019BA34208D3AB4204D0104901A8D2
:103400000195FFF7F9FE01203EBD0E4C2368200018
:10341000019308F03DF9019920000139019108F06C
:1034200017FA80235B01E418074B9C42EED104227B
:10343000034901A80195FFF7DFFE0020E4E7C0463D
:103440005555000000C007110000081130B589B0C3
:1034500008F06EF910226946254808F061FA254BFC
:10346000009A9A420ED1019B029A0F2B33D8002169
:1034700001240698013B08D2002900D00292029B49
:10348000013331D10023029325E0551CF2D1020013
:103490002100EFE710341022200004A908F040FAC0
:1034A000029B013301D1069B0293882304995B059B
:1034B000C918059B06981A03120B049105928142C4
:1034C00003D02B4201D108F053F8019B013B01933B
:1034D000019B002BDED1029B002B03D004930498A8
:1034E0004168084709B030BDE025014C2D03EFE7E6
:1034F0000000011150485936F7B50F4F0F4BFA6DC8
:1035000004001A4084235B001343FB65030010335F
:10351000019300252E00112008F072F90322BB6EE2
:103520001340AB4002351E43202DF4D1019B40C413
:10353000A342EED1F7BDC04600F0004000FEFEFF02
:10354000802270B5AD4CAE4BD200002120001C6033
:1035500008F0F6F82300AB4A88331A60AA4B1A78B1
:103560006E23002A00D01133E3620A232365A74BA0
:103570001878A74BA0630138E361C3B2032B01D8CD
:1035800010232362A34B37226361C823DB00A361AE
:1035900023008C331A60082336210F3AE518E163C3
:1035A00023646264E9670439251DE96725003B2629
:1035B000BC352E602500C0352B602500C4352A603F
:1035C00025000636CC352E602500083EC8352E6015
:1035D0002500D03529602100D4310B602100D8317D
:1035E0000A6021000225E0310D6025004221DC3512
:1035F000296025001B3EE4352E602500E8352B6050
:103600002500EC352A6022000525F43215602200E1
:10361000F032116022001831903211602200943291
:10362000136023003C2298331A60AF23DB00236031
:10363000794B2363032805D807F0EAFE33023537B8
:103640001523636096232100FA225B00A360E360E8
:10365000C8332361714BFC319200A3640A6062623B
:103660006F4A704DA2627322E2656D3A6265A2658F
:103670000232E5644A600221616696218900A166F2
:10368000626709210022E166A2676749674A684EBE
:103690002167E2673560032811D807F0B9FE960864
:1036A0009EA61023CDE70E23CBE70C23C9E720000D
:1036B0001A259C30056020000735A03005602000E9
:1036C000A83003602300FA20F8338000186023003C
:1036D0006420A433186023005F38AC3318602300E3
:1036E0000338B03318602300C630B43318602300A9
:1036F0000020B833186023003825FC339D604D4D01
:103700005A665D644C4D9A64DD619625AD001D627C
:103710004A4D9A675D62F53DFF3D9D621E25484A10
:10372000DD6618675867D9651966DA67BE23C02158
:10373000444A5B00E250444B4900635004316250FC
:10374000C4225200A350FA23E4205B000432A350A9
:103750000432A3503D493E4A3E4BD1603E49800071
:1037600019503E49E938FF3819503D490430195085
:103770003C491038D1613C4911633C4951633C4993
:1037800011603C49195019003B48F83108603B4929
:10379000D16582213A4A89005A501A0039490832C3
:1037A000D1671A003849B43211608821374A89003C
:1037B0005A501A00364988321160364ADA6407F0E6
:1037C0006FFF012008F09CF870BD200014259C308C
:1037D000056020000435A03070E7200010259C30E3
:1037E000056020000335A03068E720000E259C30DE
:1037F000056020000235A03060E7C0460004FF1FCE
:103800004866FF1F4071FF1F0846FF1F4A0AFF1F3F
:103810003A07000080C3C9019A02000050C30000AB
:103820006A180000280A0000204E000088130000DB
:10383000F009FF1F001F001168100000C4090000FC
:10384000DC05000040420F0010270000FD1BFF1F99
:10385000FC00FF1F0000FF1F092FFF1F3132FF1F59
:10386000C930FF1FDD1FFF1FF91FFF1FA521FF1F0D
:10387000491FFF1FC928FF1F712CFF1FD918FF1FE9
:10388000D527FF1F3D25FF1F4925FF1F491EFF1F8D
:10389000011FFF1FC11DFF1FF7B50B0CFF270122E2
:1038A000009300233C001E001D009446019089B245
:1038B00062469A401000084018413618B6B2FF2FF1
:1038C00002D1012E00D19FB2009802401A41AD18DA
:1038D000ADB2FF2C02D1012D00D19CB20133102BCF
:1038E000E6D10320012E07D1012D04D1019B240133
:1038F000E4191C700138FEBD102EFCD10238102DC9
:10390000F9D00230F7E710B5064C2378002B07D129
:103910000548FFF7F1FD0548FFF7EEFD0123237091
:1039200010BDC0460866FF1F1C66FF1F0C66FF1F08
:10393000F0B58BB00D0001230190102936D8FFF7A8
:10394000E2FF00231A001B48C15C01335218102B00
:10395000FAD1023B002A29D0174B184C1F680023CC
:1039600006A9E25C1600FA5C56405E540133102B47
:10397000F7D102AA07F0BCFF2A0002A9019807F0BC
:10398000A7FD07F07DFF23681B18236007F078FF71
:1039900063681B18636007F073FFA3681B18A360BC
:1039A00007F06EFFE3681B18E360002318000BB0FC
:1039B000F0BDC0461C66FF1FA844FF1F0C66FF1F1A
:1039C0000223F0B501245F4D5F4E2B705F4B91B029
:1039D0001C705F4F0393336808207B7006F052FA27
:1039E0000023984205D07A78552A02D0332A00D095
:1039F0009CE03360002006F0C5FC07F019FDFFF7DE
:103A00009FFD07F06DFD1F2201240021514B10AED8
:103A10001A70514B1C70514B1970514B19689143DE
:103A2000163A0A431A60602219689143403A0A43E1
:103A30001A6007F0F5FE07F093FFC120FF21494B04
:103A400080001A588A431A50C52292009858884319
:103A5000BF39014399509858434908408021C90112
:103A60000143802099509958C0050902090A014371
:103A7000995080213D48490107F012FF032322009D
:103A80003B49019400933B4807F0AAFC2C223A4999
:103A900005A807F06DFD05AC61782078023406F0CA
:103AA00011FAA642F8D10121002006F01FFB0121E6
:103AB000092006F01BFB314B314A196803201140E5
:103AC000A022D2020A431A608022196892040A4393
:103AD0001A6019682B4A1140802292030A431A6027
:103AE000294B2A4A934200D8012007F0C9FC07F06D
:103AF000B7FC07F095FD287807F0F2FB039B1878D8
:103B0000C0B207F0ADFD07F063FE2149042007F0C5
:103B10000FFC06F003FC00F0AFF800F0CFFD00F062
:103B200061FE00F019FA002011B0F0BD00932100F1
:103B3000174A042007F0FCFE8023DB059C62FFF798
:103B400085FC57E74A0AFF1F34F000400846FF1F74
:103B5000A463FF1F480AFF1F490AFF1F680AFF1FCF
:103B6000BCF0004000E100E0FF00FFFF0C46FF1F3B
:103B70009058FF1F0C56FF1F70B9001114F0004041
:103B8000FF7FF8FFFFFF9FFF4071FF1F0080FF1FB7
:103B90003B00010870B500252849294A29484D6392
:103BA00008CA1B051B0DED188242F9D10022264BD5
:103BB0008B63264B08211A628022254B9205DA6717
:103BC000244BDA688A43DA60234A1278012A03D048
:103BD0009A6822490A409A600121EE242048E400B4
:103BE00002686C438A430260DA6811208A43DA6013
:103BF00007F0DEFB112007F08BFE112007F0D0FB51
:103C0000184A200C0400642390420AD8FA220023A8
:103C1000D200904205D9144B0A21C01807F0D0FCFD
:103C2000C3B2124A1372124BD4801B78002B04D1FA
:103C3000104B1021187807F073FD70BD000005408F
:103C40008805054000060540FF01000000F0004027
:103C500004E100E03CF000404A0AFF1FFFDFFFFFE5
:103C600000380040B70B000030F8FFFF8C63FF1FE7
:103C7000C865FF1FC463FF1F002210B5110011208B
:103C800007F06EFD10BD0000F8B5002301250826E1
:103C9000394F3A4C3B62E3681120AB43E360E36881
:103CA000B343E36007F034FE112007F081FB1120DD
:103CB00007F04EFD40232268290013432360802330
:103CC0006268DB02134380226360A368072013430A
:103CD000A360A3682A4A1340A3608023A2689B01C3
:103CE00013431022A360236C93432364236C2B4360
:103CF000236480235B003B62226B224B1A402263C9
:103D0000626B1A406263A26B1A40A263E26B1340BB
:103D1000E3631D4AE3681340E36006F0B9F9290044
:103D2000072006F0E3F98021184A1120536C0B4359
:103D3000536407F075FBFD21154B164A89005A5054
:103D40008023C720626B5B0313436363E3688000D7
:103D50003343E360E368104A1D43104BE560195894
:103D60001140802212020A431A50802292051A60E2
:103D70000B4B5E63F8BDC04600F000403CF00040D5
:103D8000FFFFDFFFEFFFEFFFFFFF7FFF0038004087
:103D90000000FF1F953B0011FF00FFFF00E100E066
:103DA0000000054030B503A804880B20002C0ED17C
:103DB0004968074D08784978090201430A20A94259
:103DC00005D1012120001980024B1B7A137030BDF0
:103DD000192A00008C63FF1FF7B5150008AA168882
:103DE0004A680F4F14785278120222430A24BA42CA
:103DF00014D10122DBB2019200962A0007F0DEF90D
:103E0000041E0BD1074B1B68002B07D068782A785B
:103E10000002104342425041013098472000FEBD4D
:103E2000022900001063FF1F30B50125037904004B
:103E3000BFB02B4212D00A49408806F02BFD284221
:103E40000CD06A46074B69465B8D55801380064B44
:103E500060881B7A1371002203F0FCFD3FB030BD77
:103E60000863FF1F4842FF1F8C63FF1F10B5054901
:103E7000054806F0C5FC0421044A054806F082FC0A
:103E800010BDC0460863FF1FFFFF00009CB9001172
:103E90004842FF1F10B5024804F05EFC10BDC0464A
:103EA000293E0011062310B5837010330371443B83
:103EB00043712A3383714433C371002302220121E9
:103EC00003720E4B027041701C8881724472197A21
:103ED0000273C1729A784273DA7882730322C273D2
:103EE0001A7902745A7942740C2282749A79C274D3
:103EF000DB7903751123C370152010BD8C63FF1F80
:103F000010B5142007F0D4FA124B142200211860C7
:103F100007F016FC002007F09BFA012007F0E0FCF8
:103F2000022007F0F5FB032003F0BAFE042005F0A1
:103F3000CFFE052003F0F8F8062003F0C5FD0720AA
:103F400001F05AF9082006F0FDFB092000F03CFFC3
:103F500010BDC0461463FF1F10B507F071FA0120B1
:103F600007F04EFB07F08CFB002010BD094B10B58D
:103F70000400984205D0012904D12000064906F02A
:103F80003FFC10BD0229FCD1013904F0A3FB00283D
:103F9000F3D0F6E7FEFF00003A63FF1F70B50D7A1D
:103FA000100004AA2C00168810221440154220D1BB
:103FB000002E20D10A78022A18D14A685178157843
:103FC0000E4A09022943914205D00D4A914209D077
:103FD0001C800A2404E014220A491A8007F0C8FA57
:103FE000200070BD0C2208491A80F7E71C800124CC
:103FF000F6E70824F4E70B24F2E7C046F3FF0000DD
:10400000F4FF00008C44FF1F7CBA001110B50400BF
:104010000749084806F0F4FB074804F0DDFA0020E1
:10402000E40704D50721054A054806F0ABFB10BD9F
:104030003A63FF1FFFFF00006D3F0011E0B9001160
:104040008C42FF1F00B50C4BBFB01A780B4901A87A
:1040500000F0FAFB6B4680B25880002809D06A460F
:10406000074B69461B881380064B0022188803F013
:10407000F1FC3FB000BDC0461863FF1F1963FF1F6E
:10408000E642FF1FEE43FF1F00B50C4BBFB01A788E
:104090000B4901A801F024FC6B4680B2588000282F
:1040A00009D06A46074B69465B8D1380064B002298
:1040B000188803F0CFFC3FB000BDC0464263FF1F2D
:1040C0004363FF1F8C42FF1FEE43FF1FF7B50E0037
:1040D000377A1C0008AB11003D001A8820231D40D0
:1040E0001F423CD13378022B3BD173681F785B7839
:1040F0001B023B431E4FBB4208D01E4FBB4214D095
:104100001D4DAB4221D00A252800FEBD002A2AD130
:10411000142C2AD82200F06807F02AFA174B1C70DA
:10412000012CF1D9FFF7B0FFEEE7002A1BD1202CBC
:104130001BD82200F06807F01BFA114B04211C70F9
:10414000104B187807F0ECFADEE7E3B20124009296
:1041500001940A00310007F031F80500D4E7082582
:10416000D2E70125D0E70B25CEE70D25CCE7C046E9
:10417000F3FF0000F4FF0000022900004263FF1F6C
:104180001863FF1FC463FF1F332310B504000370BF
:104190000A220749013007F0EBF9064B0F201B6894
:1041A0001A0AE37222731A0C1B0E6273A37310BDFA
:1041B0008C63FF1FB463FF1F30B501250379040032
:1041C000BFB02B4213D00B49408806F063FB284256
:1041D0000DD06A46084B01A81B881380FFF7D4FF57
:1041E0006B46588000226946608803F033FC3FB07C
:1041F00030BDC0463A63FF1FE642FF1F10B50248BC
:1042000004F0AAFA10BDC046B941001170B51600FD
:1042100004AA148805AA15784A6850781178000213
:104220002A4A0843801805284BD807F0F1F80313F1
:104230001E29343F0720042C0BD80522121BAA424A
:1042400000D92A0022491A803000091907F090F994
:10425000002070BD0720112CFBD81222121BAA428D
:1042600000D92A001B491A80EEE707200E2CF0D84F
:104270000F22121BAA4200D92A0017491A80E3E72D
:104280000720032CE5D80422121BAA4200D92A00D9
:1042900012491A80D8E70720032CDAD80422121B0F
:1042A000AA4200D92A000E491A80CDE70720032C24
:1042B000CFD80422121BAA4200D92A0009491A8029
:1042C000C2E700220A201A80C3E7C046DCD5FFFF00
:1042D0002BBA00116063FF1F1BBA001116BA001140
:1042E00011BA00110CBA001110B50D21024A034891
:1042F00006F048FA10BDC04600BA0011FC42FF1F8C
:10430000F0B50024274E85B03000B47100F0E2F81B
:10431000254D264BEA89297C9A422FD1042330006F
:1043200003AA00F057F90400300000F011F901234E
:10433000B371002C34D16B4699892B68C9BA4B43B1
:1043400029891B4A1B145B1853806B46D9896B68FB
:1043500049BA89B24B4369891B0C5B181548191C73
:104360001BB2834200DD011C0B0400D50021138821
:10437000918001331380200005B0F0BD0227220098
:1043800003AB3000009700F0F7F80E230400297CFF
:104390000122300000976B4400F0EEF80443C3E7BD
:1043A0001C00E8E7D443FF1F7463FF1F8305000070
:1043B0008C63FF1F0F27000073B5234E300000F001
:1043C00089F8224D07236A463000297C00F002F963
:1043D00004003000002C33D16B461B787F2B2FD884
:1043E00000F0B6F86B46D878F02302041B031A409D
:1043F0006B469B8816495BBA9BB21A432B6800092F
:1044000053432A891B0C9B184B806B465A789B7828
:1044100012031B011A436B68024353436A891B0C46
:104420009B180C481A1C1BB2834200DD021C1304AB
:1044300000D500220B888A8001330B80200076BDD6
:1044400000F086F80124F9E7D443FF1F7463FF1FCF
:104450008C63FF1F0F27000070B5114C237C002BCD
:104460000FD0382B0ED10F4D280000F033F8CC239D
:10447000AC222800217C9B0100F0F4F8280000F019
:1044800067F870BD084BE2899A42FAD1054D2800C1
:1044900000F020F800222800217C00F0C5F8EDE7AC
:1044A0007463FF1FD443FF1F8305000010B5084B42
:1044B0001A7C002A09D05B69002B06D09847041E9D
:1044C00001D0FEF79DFD200010BD0124F9E7C04694
:1044D0007463FF1F70B5C17905000C00631E9C4119
:1044E0001A4BE402E41849000460C9B2007905F0EF
:1044F00033FEE979687949000131C9B205F02CFE33
:10450000E8790930C0B207F023F90023E36661338C
:104510002360AA795B3B002A0ED022689A43023BB3
:10452000134323600A23E3610733236200232363D9
:10453000A3630133E36370BD22689A4302231343EC
:104540002360462363610633A361EFE70050004018
:1045500070B5002504000368DD66C0790930C0B27B
:1045600007F0D6F92900207905F092FD290060793D
:1045700005F08EFD70BD0000F8B51E0006AB1D787D
:10458000002304681700E366616007F0D1F8012397
:104590008022E3662B0027615200013B08D207F01E
:1045A00087F808200A4A1168002D03D12800F8BDB9
:1045B0002261F2E7236F034203D02369013D337088
:1045C000013613685B1A032BEED90125EEE7C046CE
:1045D0006008FF1F70B51C00002305681600EB661D
:1045E000696007F0A5F801238022EB6623005200E2
:1045F000013B08D207F05CF808200A4A1168002C39
:1046000003D1200070BD2A61F2E72B6F034203D073
:104610002B69013C3370013613685B1A032BEED90A
:104620000124EEE76008FF1F002370B50468150041
:10463000E366616007F07CF80123E366256107F01B
:1046400037F88020064A80001168636B034205D169
:1046500013685B1A032BF8D9012070BD0020FCE71A
:104660006008FF1F70B51D00002304681600E36694
:10467000616007F05DF80123E36626610F33626B2A
:104680001A42FCD02B0A23611023626B1A42FCD021
:10469000EDB2256107F00CF88020074A8000116810
:1046A000636B034205D113685B1A032BF8D9012011
:1046B00070BD0020FCE7C0466008FF1F10B5084C25
:1046C000E368002B08D1074B1B685B045B0C0A33C3
:1046D0006360054B1B68236007F082F8A06010BD83
:1046E000B463FF1FC8F00040CCF0004010B507F0E5
:1046F0001FF80F4B996A9A6A8A42FBD10D4C626887
:10470000A0688A18121A531E884200D31300A160B1
:104710002168DA0B52185B0407495B0C6360226066
:104720000B60064B1A6006F0C3FF206810BDC04640
:1047300000F00040B463FF1FC8F00040CCF0004020
:1047400070B51F4C23793F2B01D93F2323711D4B9B
:1047500022791A701878C0B207F0B2F818231A49F3
:104760001A4A0B801A4913800B805380A379194988
:1047700080200B800C21938001334B430001191CD6
:10478000834200D9011C144BD18019806379002B1E
:1047900011D101336371237A012B01D802232372D3
:1047A0006279237A0D4853430A21584306F008FFE3
:1047B0000B4D286070BDA02BEDD9A023EAE7C046C1
:1047C000A863FF1F480AFF1FEC43FF1FB445FF1FEC
:1047D000EA43FF1F9465FF1FE843FF1F71020000BB
:1047E0009863FF1FF8B513210020FEF7F7FD114C69
:1047F000011E114D09D10C22104BC1CBC1C42800A0
:1048000006F09EFFFFF79CFFF8BD0C2220000C492C
:10481000FEF7B8FD0C2802D0084B43CB43C40C2252
:1048200028000849FEF7AEFD0C28EBD00C22002131
:10483000E5E7C046A863FF1F7463FF1F70BA00114D
:10484000FC0C0000F50C0000F0B5002504000E0083
:1048500085B0AA4263D04B1C087801934B788978C5
:10486000377909021943F3783F061B040B431F43B2
:10487000039720706570252800D173E012D81028A6
:104880000AD806F0C5FD46E52C2C2C87958E2C2CDD
:104890002C2C2C2C2C2CC500232800D1A7E0FF2386
:1048A000637094E0562857D010D8332800D199E08F
:1048B000552837D02628F2D1934B2900132218000F
:1048C0001D0006F03DFFFEF79BFB5AE0722800D169
:1048D0007FE0DC2800D1DAE0712800D16FE0DB282E
:1048E00000D0EFE0042ADAD91025052A05D0551F9B
:1048F0002A003800711D06F03BFE05223100200021
:1049000006F036FE2A003900601D06F031FE05353E
:1049100005E00C2220007D4906F02AFE0C25280027
:1049200005B0F0BD013A7A4D0C2A13D8002A0AD0FE
:104930002800019906F01CFEFFF702FF0C22280058
:104940007449FEF759FC29000C22601C06F010FE89
:104950000D25E4E70C22EBE76D4D6F4B2A0043CBAE
:1049600043C2E9E7013A684D0C2A11D8002A08D061
:104970000199280006F0FCFD0C2228006749FEF78B
:104980003BFC29001322601C06F0F2FD1425C6E74B
:104990000C22EDE705226249601C06F0E9FD0625C0
:1049A000BDE712225F49601C06F0E2FD1325B6E761
:1049B00008225D49601C06F0DBFD0925AFE7717830
:1049C000F72900D96BE7594B188801F0E5FB022560
:1049D000A5E7574B012A03D072781A706270F6E788
:1049E0001B785DE72000FFF7CFFB050097E7042A5F
:1049F00004D9504D2F6006F0F3FEA860FFF776FE55
:104A00000422039003A9601C06F0B2FD052586E789
:104A1000494D062A15D906222800019906F068FE9C
:104A200000280ED006220199280006F0A1FD0622DA
:104A300042492800FEF7E0FB01233D4A11780B4371
:104A4000137029000622601C06F092FD072566E718
:104A5000931E3B4F1A2B04D87378002B09D100F01A
:104A600027F9384B39001D78601C6A1E06F080FD5E
:104A700055E7551E2A000199380006F079FD3249A4
:104A8000AAB23800FEF7B8FB00F048F9E9E7022ABD
:104A900000D804E77378BFB26370B378A370032AB9
:104AA00005D0033A390092B2F01CFEF7A5FB1022A4
:104AB0003900E01CFEF766FCC51C002800DB2EE771
:104AC000607084E7DA2800D0E9E6042A00D8E6E638
:104AD000082A15D9B37972791B021343F2791204AB
:104AE0001A43337A1B0613433B603B6805223100AF
:104AF0002000039306F03CFD0422601D03A95AE741
:104B0000FE236370F1E7C0467463FF1F7CBA001197
:104B1000A863FF1FFC0C000070BA0011F50C000028
:104B20008063FF1F6063FF1F2845FF1FEE43FF1FC9
:104B3000A463FF1FB463FF1F6509FF1FADAC000036
:104B4000A765FF1FA565FF1FAEDE000070470000D0
:104B5000020010B5094B0A32094C92B2DA815A822E
:104B600098811882207802F07DF90422054B0121FA
:104B700020781A7006F0D4FD10BDC046B244FF1F65
:104B8000F265FF1FF165FF1F013870B5042809D8D1
:104B900006F03EFC0309230812001E4B0221187880
:104BA00006F0BEFD70BD1B4B0821187806F0C8FE4C
:104BB0000022194B1A72F5E780220024164B154D7E
:104BC00052001A81082128781A68DC7206F0E8FC85
:104BD0002100287806F0BCFBE4E70E4B082118788A
:104BE00006F0AEFE0D48FFF75DF90D4B0D4A9B79BF
:104BF00093800D4A13800022074BDA720132FF3294
:104C00001A810A4B1B78002BCCD0094A136006F09E
:104C1000BFFBC7E7C463FF1F9863FF1FF743FF1F76
:104C2000A863FF1FB445FF1F9465FF1FA463FF1F08
:104C300034F0004010B5002905D1082803D1013116
:104C4000013005F053FA10BD10B501290FD1082825
:104C50000DD10021013005F049FA054B1B78002BDE
:104C600005D02622034B04485A72FFF771FF10BD8E
:104C7000C865FF1F9863FF1FC40900000300F0B55B
:104C80000A4D8E18B14202D152008018F0BD0C7846
:104C90002F6824093C5D0F271C700C7801313C40C3
:104CA0002F683C5D5C700233ECE7C046E443FF1FB5
:104CB0000E22114B10B51A700D23104C10492370A1
:104CC000093A043B0F48637006F052FC2D23012281
:104CD0000D490E48E371FFF7D1FF01220C49FFF7A0
:104CE000CDFF01220B49FFF7C9FF00220A4910003E
:104CF000FEF782FA10BDC046C465FF1FA565FF1F01
:104D00002BBA0011A765FF1F6709FF1FAD65FF1FC5
:104D10006609FF1F6509FF1FAEDE000070B5124C6B
:104D2000132220001149FEF72DFB114D002817DD3D
:104D3000AB78002B14D0431C2B7009236B7000231D
:104D400000190370287829000130C0B206F018FC61
:104D5000297822000139C9B2002005F031FC70BD6C
:104D6000FFF7A6FFEEE7C046A765FF1FAEDE000017
:104D7000A565FF1F10B5114B1A781870002A0ED0C8
:104D800000280BD10E4B1A78062A07D85423D3409B
:104D9000DB0703D50B4B187802F064F810BD002830
:104DA000FCD0074B1B78012B02D0033B022BF5D81C
:104DB000044B0121187806F0B3FCEFE7C865FF1F2C
:104DC000F165FF1FF265FF1F70B5504E504A514903
:104DD0003070082005F080FA0121092005F086F9DD
:104DE000092005F067FA0121002005F07FF9002075
:104DF00005F060FAFEF704F906F092FB032246493B
:104E00004648FFF73BFF2D24030004221C70444951
:104E10000130FFF733FF30230470424D424C4370A2
:104E200083702E3B062220004049EB87FEF7AAFA4A
:104E3000062813D0200006F05BFB022809D00321CE
:104E4000200006F06DFA8D23E3706E3B2371193359
:104E50006371062220003549FEF7CEF9344B1B68FA
:104E6000FC335C64FFF75AFF0020FFF783FF314CEF
:104E7000314A0121314B1278207801F0B5FF304AD8
:104E8000304B12780021207801F0AEFF01222E4B2A
:104E90001A702E4B5B78552B31D12D4B3B325A7209
:104EA0002C4B2D4AAB81EA812B826A8220213078FB
:104EB00006F06EFC0120404205F0CEFB012040428E
:104EC00005F06AFCFFF710FAFEF7D0FF00F0A0FC37
:104ED00001204042FFF79AF8012006F0B1FCF720CC
:104EE00001F03EF90121307806F01AFC307802F02A
:104EF00015F91A4806F07CFAFEF7C6FE70BD64226A
:104F0000174B5B7953431A000A32CBE7C463FF1F88
:104F1000354C0011494C00112845FF1F6063FF1FED
:104F20008063FF1FB244FF1F6509FF1FADAC000087
:104F30004866FF1FF265FF1F1644FF1FF743FF1F60
:104F4000C465FF1FA565FF1F9665FF1FA463FF1FB4
:104F50009863FF1FC4090000CE090000C663FF1F4D
:104F6000A863FF1FF8B50A0020230D001A4019425C
:104F700051D0544B1B78002B3CD0FFF7B7FB524B62
:104F8000524C534E99686268737A8A1ADB039A42CC
:104F900002D36160FEF778FE327A217A531EDBB2CB
:104FA00099422AD1FFF758FA637A002B1FD0013BB0
:104FB000DBB26372002B1AD1464B5B78552B01D1C3
:104FC00006F0E6F9E37A002B0CD00023424A434F67
:104FD000E3721388380001331380FEF763FF390052
:104FE00006F08EFB642370795843FFF7B1FD237AF6
:104FF0000133237220206840F8BD9142D4D30023AE
:105000002372FFF753FA354F3800FEF74BFF390094
:1050100006F076FBC8E70BB2002B0ADA304B1878A3
:1050200006F0BEFB002801D006F0EAF9802000025D
:10503000E1E70224214206D0244B01201A72FFF737
:1050400099FE2000D7E70B071BD5FFF74FFB1E4B40
:105050001E491F4C98684A68637A821ADB039A4299
:1050600002D34860FEF710FEFFF720FAFFF7F4F9CD
:1050700000F0E8FB2368DB0701D5FFF7BFF8082045
:10508000B9E710240E002640214206D00D4B1B78B4
:10509000002BD6D1FEF7FEFED3E70124214209D032
:1050A000104800F06DF806F04BF93100092005F0CA
:1050B0001DF8C6E704240800204021429CD0FEF7DA
:1050C000C1FFBEE7C865FF1FB463FF1F9863FF1FE2
:1050D000A863FF1FA463FF1F8C63FF1FF743FF1F1D
:1050E000C463FF1FDC43FF1FF0B51B4B1B4F1B8826
:1050F0003A8804001A4E1B4D85B09A420DD832886A
:105100009A420AD3184B1A882B889A4205D1174A1B
:10511000174B12881B889A421BD0052001F076F8A5
:105120003B8802AA13803388019053802B88114D4D
:1051300093800F4B02A91B88D3800F4B2A781888C5
:1051400002F092FD0D4B08212878019A1C7006F0A0
:10515000EFF905B0F0BDC0469265FF1FEC43FF1F9D
:10516000EA43FF1F9465FF1F9065FF1F8E65FF1FB9
:10517000E843FF1FF265FF1FEE43FF1F8C65FF1F13
:1051800013B50C4B1C78002C11D1002801D00A4B10
:1051900018600A4A0A4B11780A4A10780A4A0192A2
:1051A0000A4A0092002205F003F9200016BD1124DE
:1051B000FBE7C046F165FF1F8865FF1FF065FF1F15
:1051C000E065FF1FF265FF1FCC65FF1FD065FF1F65
:1051D00010B5064B12201B78052B06D1044B132269
:1051E0001988044B187801F0EDF910BDF165FF1F27
:1051F000EE43FF1FF265FF1F10B500240122114B83
:1052000052421870104B1C70104B1A8001F086FF30
:1052100004220F4B21001A700E480C3206F0D8F809
:10522000102221000C4806F0D3F807220B4B1C601B
:105230000B4B1C700B4B1C700B4B1A700B4B1C70E8
:1052400010BDC046F265FF1FF165FF1FEE43FF1F53
:10525000F065FF1FE065FF1FD065FF1FCC65FF1FD6
:10526000A465FF1FA365FF1FF043FF1FA265FF1F7B
:10527000F8B5174C0600257806A814240078052DEB
:1052800023D1B41F134FA5B21824BD421DD88D1FC2
:10529000ADB2BD4219D8FA256D00AA4215D21D0043
:1052A0000D4F0A3DADB2BD420FD80C4C26800C4CC0
:1052B00021800C4900240A800B4A1380FFF714FF59
:1052C0000A4B0421187806F03BFB2000F8BDC046CD
:1052D000F165FF1F790C0000750C0000EC43FF1F07
:1052E000EA43FF1F9465FF1FE843FF1FF265FF1F9E
:1052F000F0B50BB20D0089B0002B00DB70E1A44EBD
:10530000307806F04DFA041E50D00378A22B00D15D
:1053100022E1D02B1AD0912B45D143780E2B42D1CC
:105320009C4B82889A423ED19B4A83681278052A18
:1053300039D1032018567F2835D0984B1B68002B95
:1053400031D05B68002B2ED098472CE0807807285E
:1053500029D806F05DF80428183F3F74A8D8637870
:10536000002B0CD101218C4B19708D4B1A78002A1F
:105370005BD08C4B307801F037FD002855D00722E8
:10538000854B1A7051E061780029F8D1E378002B41
:1053900011D0854A854B1278307801F025FD607078
:1053A0006378002BEBD1200006F02AF88020000261
:1053B000684009B0F0BD784B1B78022BF3D0012177
:1053C000307806F035FA0028EAD10121307806F06D
:1053D000A7F9E5E76378002BD1D16F4F032807D1F8
:1053E0003B78052B02D101333B701EE00223FBE723
:1053F0006F4B1A886F4B0293002A0BD01B78002B3F
:1054000003D00121307806F093F83B78062B04D1C5
:10541000013BE9E7029B1A70F7E7042B41D1012118
:10542000029B3078197006F07BF95C4B1B68002BEF
:10543000B9D01B68002BB6D0574A107884E7637840
:10544000554F002B27D10622211D5B4806F090F80E
:1054500062895A4B5A491A80A2895A4B1A80E389A9
:105460000B800521397058490A80584A1380228AD6
:10547000574B1A80574B1B78012B09D11F2000F086
:10548000C5FEFA22920042430421307806F050F81B
:105490000022484B75E7312B00D070E70022454BC6
:1054A0001A700323A0E706220021434805F090FF6D
:1054B0000023454A04211380444A30781380444A2B
:1054C000138006F03DFA0821307806F039FAA37906
:1054D000083B5A425341304A03331370304B1B7818
:1054E000002B06D0334B30781A78002A06D001F012
:1054F000B9FC0122314B52421A8096E70121197002
:1055000006F00EF9F5E70821307806F019FA63780D
:10551000002B00D047E72C4B2D4F0293E388029AD3
:1055200004211380294B307803932389039A138035
:1055300063893B8006F07CF9002800D033E7264BD6
:105540001B68002B00D12EE7039902983A8809883E
:1055500000881B68984726E74379132B00D022E781
:105560000389012B0AD11D4B1B78022B06D1082180
:10557000307806F0E5F9FFF72BFE14E7052000F080
:1055800045FE08210200307805F0D2FF0BE7C04647
:10559000F265FF1F05140000F165FF1F8865FF1FFE
:1055A0001644FF1FF743FF1FC465FF1FA565FF1FBC
:1055B000C665FF1FC865FF1F9765FF1FEE43FF1FEE
:1055C0009E65FF1FA065FF1F9265FF1F9065FF1F6F
:1055D0008E65FF1F9665FF1F8465FF1F8C65FF1F8B
:1055E0008020C001014200D0E2E6CB0731D5324B2A
:1055F0001B78002B1DD0314E05AC3378052B1AD10A
:10560000023B23702E4B21001B7823722D4B1B78FD
:1056100063722D4B187801F08BFB002809D007200E
:105620002A4B30701B68002B03D01B68002B00D066
:1056300098470120BCE60E20254B06221B78254901
:105640002370254B1B78637002ABC01805F090FFE8
:10565000D8E7022308001840194209D0174B1B78DD
:10566000052B03D11D4B188805F04AFE02209FE64A
:105670000424214203D0FFF737FD200098E60823D9
:1056800008001840194200D193E6154B1C78012CF4
:1056900003D0022C0DD008208AE6124B124A13497F
:1056A00013481B881288098800880094FFF7E0FDE2
:1056B000F1E7FFF78DFDEEE7C865FF1FF165FF1FFE
:1056C000F043FF1FA265FF1FF265FF1F8865FF1FE4
:1056D000A465FF1FF143FF1FA365FF1FEE43FF1FDC
:1056E0008C65FF1FE843FF1F9465FF1FEA43FF1F00
:1056F000EC43FF1F10B502A804880B20002C10D12A
:10570000496808784978090201430C48814209D167
:10571000022119800A4B59881170DB7800205BB296
:10572000537010BD074C0A20A142FAD10221198002
:10573000034B998811705B79F0E7C0466E2A000030
:105740008C63FF1F6F2A0000F7B5150008AA1688A2
:105750004A680F4F14785278120222430A24BA4240
:1057600014D10122DBB2019200962A0005F026FD39
:10577000041E0BD1074B1B68002B07D068782A78D2
:105780000002104342425041013098472000FEBDC4
:10579000022900000466FF1F30B5012503790400CB
:1057A000BFB02B4227D01549408805F073F8284236
:1057B0000DD06A46124B69465B8D138002235380DD
:1057C000104B5B8893806088002202F043F90E49F9
:1057D000608805F05FF8C0070DD56A460B4B694637
:1057E0001B88138002235380064B9B88938060881C
:1057F000002202F02FF93FB030BDC046FC65FF1F0C
:105800001844FF1F8C63FF1FF465FF1F7244FF1FC6
:1058100010B5074C0749200004F0F2FF20000649AC
:1058200004F0EEFF0721054A054804F0ABFF10BD68
:10583000FFFF0000FC65FF1FF465FF1FFCBA0011AD
:105840001844FF1F10B5024802F086FF10BDC04685
:10585000995700110200F0B501270A480A4E511865
:105860008B1A002B00DCF0BD082415784308684033
:1058700038404000805B013C58406D08002CF5D159
:105880000132EDE7FFFF000016BB0011F0B5002567
:105890000F269D4200DBF0BD4C5D070944403440BB
:1058A000A400A05801357840F3E70000F0B589B0B6
:1058B0006A460D000B000F27110010351C780133CC
:1058C000260024093E40167054700232AB42F5D1D6
:1058D0002023024AFFF7DAFF09B0F0BD1CBB00111C
:1058E000F0B54E780B7889B036020C0017000190A5
:1058F0001E43012A61D9954B9E4200D877E00133BF
:105900009E421CD1062A17D1CA788B7812021A43FC
:105910000B791B0413434A7912061A438C4B5A61C4
:1059200000221A705A808B4A5A608B4A9A608B4ABE
:10593000DA60002009B0F0BD88225205EEE7884BFE
:105940009E423CD182498B78002B00D0F6E00C2A95
:1059500031D10F22A3789343E278120213432279C4
:10596000120413436279120613434B60E279A07963
:1059700012020243207A00041043627A12060243A4
:10598000CA60E27AA07A1202024376484A818342D0
:1059900008D804236E49142201980B7005F0E8FD25
:1059A0001420C7E71201D21889235B059A42F0D868
:1059B00001238B70BDE7022AFAD00523EAE76A4A81
:1059C00001239642E6D1FFF703FC052F0CD9E378BB
:1059D000A2781B021343227912041A4363791B062F
:1059E0001343624A0393136005F0D2FCA1E7584DBC
:1059F0002B78002B9DD1AB78002B00D1A0E02B8918
:105A000001339BB20093B34200D091E0132AD4D962
:105A1000CF7C8B7C3F02122120001F43FFF71AFF2F
:105A2000874200D08EE0002E3DD1E378A2781B02A1
:105A300013432279E96812041A4363791B0613435E
:105A400003930A228B4212D1FF23A370E3702371C8
:105A500063716B89002B09D1E37B227C1B0212044A
:105A60001343A27B13431B0901336B8100226B8913
:105A7000002B8ED0002A67D1686837013818000BD8
:105A80006B6900030390984205D9686105F000FE38
:105A9000EB780133EB7068681022A11C381805F010
:105AA000CFFD2E8145E76F89009A7B1E9BB2934202
:105AB0003AD1E278A37812021A43237905A81B048D
:105AC000134362796C6812061A43EB6800920392E2
:105AD000211D0C22049305F04BFD0120260004A992
:105AE00040421036FFF7E2FE013F012F17D1009A26
:105AF0000B232861824200D04CE704221C4920007D
:105B000005F09EFD042203A9686805F031FEE968EE
:105B1000039AFF23914200D13CE7F73B3AE731007B
:105B2000FFF7C4FE1036DFE70923B742A4D831E7F8
:105B3000009BB34200D9FCE607232BE7022329E7A9
:105B4000032327E7062325E70A2323E7FFFE0000B8
:105B50008C44FF1F00000111FFFF00005048593620
:105B600001FF0000FFFF001102FF000034F00040C1
:105B70009844FF1F10B5034C0B000122210000F0D8
:105B80006BFA10BD355D00110B8870B506000D0075
:105B90000224162B11D92B000322094900F05CFACC
:105BA000041E0AD1074B2A881B88191C934200D96E
:105BB000111C300089B200F0EFFA200070BDC04621
:105BC000615D00116266FF1F10B54A780400013A5A
:105BD0000B000220012A07D80A78002A04D00522E7
:105BE0002000024900F038FA10BDC0468F5D001158
:105BF0000A7810B50B0004000220002A04D0072206
:105C00002000024900F028FA10BDC0463B5E00119A
:105C10000A7810B50B0004000220002A04D00922E3
:105C20002000024900F018FA10BDC046A15E001124
:105C300010B5034C0B000B22210000F00DFA10BD33
:105C4000D15E001110B5034C0B000D22210000F0B5
:105C500003FA10BD435F001110B5034C0B000F2277
:105C6000210000F0F9F910BD9D5F00110A7810B510
:105C70000B0004000220002A04D011222000024957
:105C800000F0EAF910BDC046AD5F0011002310B569
:105C90001322190000F0E0F910BD000010B5034C0C
:105CA0000B001722210000F0D7F910BDFF5F001193
:105CB000002310B51922190000F0CEF910BD000024
:105CC00010B5034C0B001B22210000F0C5F910BDDC
:105CD00039600011F7B584890D0006000121002C00
:105CE00022D000238268D3561778002B1EDA0C2CA2
:105CF0001AD90C3CA4B2131940880093230002F077
:105D000086FE431E984101307B06DB0F6B703F23FC
:105D1000013C1F40A4B22870AF70AC80002C07D0AB
:105D2000B3680133AB6000210800FEBD0020EBE743
:105D3000AC60F8E70B7803704B8843704B881B0A04
:105D400083700B79C370042070470420022B06D1A6
:105D50000020537811781B02009A0B431380704780
:105D60000B8803700B881B0A4370022070470420C5
:105D7000009983420AD1537810781B0203430B80A9
:105D8000D37890781B02034300204B807047F8B50E
:105D90000D004B7801240021461C03702B788B42A8
:105DA00001D82000F8BD6B78B01C4F1C012B10D11E
:105DB000890069184B88022233704B88B9001B0A8E
:105DC0007370691805F084FB04360434A4B2F9B288
:105DD000E4E7122359436B185A88043132705B8808
:105DE00010221B0A7370691805F072FB1236123408
:105DF000ECE770B5049D14001E00052B01D80420AB
:105E000070BD637812781B0213432B80E378A2786D
:105E10001B02134302226B802A71211D681D063E5E
:105E200005F056FBB2B22A81F02AE8D82800A11D5D
:105E30000A3005F04DFB0020E2E7002310B50A7898
:105E40009A4201D8900010BD9A008A1854880133F4
:105E500004705488DBB2240A447094888470928859
:105E6000120AC2700430EAE710B51100029C062B3A
:105E700004D004201022142B01D010BD0222227164
:105E80004B7808781B0203432380CB7888781B0269
:105E9000034363800431601D05F01AFB0020ECE72A
:105EA00010B50C788B7804315C43E4B203702200A7
:105EB000013005F00DFB601C10BD0420022B06D143
:105EC0000020537811781B02009A0B43138070470F
:105ED00010B50C000A88023105F0FAFA208810BDCE
:105EE00070B504000D0004981100012B01D80420A6
:105EF00070BD167852781202324302800200F832E6
:105F000055701470E825002C00D10C35023B9AB274
:105F10004280AA42EBD80231043005F0D9FA0020C1
:105F2000E6E70420009983420AD1537810781B02D7
:105F300003430B80D37890781B02034300204B80EF
:105F4000704710B50C000A88023105F0C1FA2088AC
:105F500010BD000070B501211E000420049C0E40FD
:105F60000B4218D1CB40DDB28D4214D90A49DBB2C5
:105F7000098899420FD32300F6331D70330058006F
:105F800011184978165C0902314301332152D9B204
:105F90008D42F4D8002070BDAC44FF1F10B50C003A
:105FA0000A88023105F094FA208810BD10B50C78EB
:105FB0008B7804315C43E4B203702200013005F0B9
:105FC00087FA601C10BD10B511000298032B01D890
:105FD000042010BD14785278043B12022243028040
:105FE000CA788C781202224342809AB28280F22AC6
:105FF000EED80431063005F06BFA0020E9E710B561
:106000000C000B8803700B881B0A43704B8883704D
:106010004B881B0AC3708A880430063105F058FA91
:10602000A088043080B210BD0420012B03D10020D1
:106030001378009A1370704710B50C000B8803702A
:106040000B881B0A43704A880230043105F040FA7D
:106050006088023080B210BDF0B589B003931E4B4A
:10606000029242000700D05A019102F020F8132555
:10607000061E2DD0029B01240370019B002B04D02F
:10608000001903999847001984B26B461B7A5BB2DA
:10609000002B0FDA1021380002F01CFB1925002814
:1060A00013D130003219E1B202F066FC051E0CD1AA
:1060B0000C34A4B2042304AA380005A993800696E0
:1060C000948101F0AFFD051E02D0300005F040FCC8
:1060D000280009B0F0BDC0466066FF1F70B505001E
:1060E0000C0000280CD00020814209D01022200092
:1060F000044905F0EDF901202B7823736B78637365
:1061000070BDC0465CBB0011F0B506000D00170065
:106110001C0085B002291BD00020102907D1022BBA
:1061200007D0102B03D115E00020102C08D005B0AB
:10613000F0BD69463800FFF7D1FF2A0069460BE041
:1061400069463000FFF7CAFF22006946380004E0C4
:10615000022BE9D12A003900300005F0D9F9E6E731
:10616000031CF72800D9F723032008499AB2013A03
:106170000B80D317034006499B189B100B80D30F4D
:1061800004499B185B100B807047C046B044FF1F4A
:10619000AE44FF1FAC44FF1F034B1B888B4202D34E
:1061A000024B4000C1527047B044FF1F6066FF1FA2
:1061B000014B4000185A70476066FF1F1722014BC1
:1061C0001A8070476066FF1F70B505000E2005F04D
:1061D0001FFA041E13D0D0230370002306228370FD
:1061E00007494570033005F073F9064B2100DA8A40
:1061F00062811B7E2373044B187805F031FB70BD60
:106200007C66FF1F6C66FF1F0045FF1F262803D812
:10621000024B4000C05A70470148FCE7B244FF1FE0
:10622000FFFF000070B506000C00094D1C22002184
:10623000280005F0CDF8074B1E70074B1C7005F0C9
:106240009FFA0123002801D0002312202B7070BD7B
:106250006C66FF1F0045FF1F8D66FF1F70B50500B0
:106260000D4C0800E260A16010220021656005F07D
:1062700027FA012803D11021A06802F058FD10224E
:106280000021280005F01CFA012803D110216068C4
:1062900002F04DFD70BDC0466C66FF1F70B5041E58
:1062A00005D1002903D006220D4805F011F90D4B48
:1062B0001D78012D11D1002C05D102221A7005F094
:1062C0007FF8280070BD00221A70074B1B78FF2B47
:1062D000F7D02000FFF778FFF3E70025F1E7C0468D
:1062E0007C66FF1F6C66FF1F0045FF1F030010B593
:1062F000002801D1002010BD00780B4A002803D1EE
:106300005988D1821B7913761378022BF2D100239E
:10631000984200D103331370044B1B78FF2B01D03C
:10632000FFF752FF0120E6E76C66FF1F0045FF1FE5
:10633000002911D000280CD04B79012803D140222C
:106340005242134303E03F221340032802D00120AE
:106350004B7170474022F4E70800FAE770B5094D29
:106360000100287800280BD0074C0622200005F0F9
:10637000AFF821002878FFF7DBFF200005F0B0F927
:1063800070BDC0468C66FF1F6666FF1F00290AD0DD
:10639000012808D13F224B799343C02B03D0403BC7
:1063A0005A425341981C704770B5174D06002B7820
:1063B000FF2B15D00A2005F02BF9041E10D0D02396
:1063C0000370C83B8370114B11491B784670C37032
:1063D0000622043005F07CF82100287805F040FA08
:1063E0000C4B1B78012B0DD10B4B1B68002B03D0E2
:1063F0009B68002B00D09847084B04211878084A66
:1064000005F0CEF870BDC0460045FF1F8C66FF1F2B
:106410006666FF1F8866FF1FB466FF1FB866FF1F12
:1064200060EA0000014B98687047C0466C66FF1F29
:10643000014BDB68186870476C66FF1F074B10B58F
:10644000DA68136801331360054B1878FF2803D00E
:106450008021C90105F064F910BDC0466C66FF1FBC
:106460000045FF1FF7B50E0002F0C8F8051E1CD04E
:106470000E4B06621F78002F00D10778AB791020F1
:10648000019305F0C5F8041E0FD0D0230380C73B4D
:106490008370019BE91DC3700622043005F018F8D3
:1064A00021003800E66005F0DBF9F7BDFE44FF1F70
:1064B000014B18787047C0468C66FF1F054B0028BB
:1064C00005D1054B1A78054B002A00D1014B180065
:1064D0007047C0467C66FF1F8C66FF1F6666FF1F05
:1064E000014B58687047C0466C66FF1F024B186826
:1064F000431E9841C0B270479066FF1F421E0300C2
:106500000120152A03D9FF3B5A425341D8B27047A4
:10651000F0B51C0000230E0085B0039002920B70B2
:10652000029A934201D3002019E0E55C5A1CD2B2D2
:10653000002DF8D0029851198142F4DC0233DFB209
:10654000A35C18000193FFF7D9FF002807D0013D95
:10655000019A0399EBB233708A4202D1E01905B077
:10656000F0BDDB19DBB2DBE710B50C0002F09EF8E2
:1065700003001220002B03D02100588804F088FF6C
:1065800010BD000070B50E4D84006359002B15D06E
:10659000186A002801D004F083FF2B59586A00289C
:1065A00001D004F07DFF2B59986A002801D004F037
:1065B00077FF285904F074FF00232B5170BDC046AB
:1065C0009C66FF1F1C4B70B504000E00150099421D
:1065D0000AD11A4B1B68002B01D1122070BD1B6819
:1065E000002BFAD09847F9E7154B994215D1134B78
:1065F0001B68002B0AD01B68002B07D09847002887
:1066000004D1104B1C70104B1D70E7E729002000CF
:10661000FFF7AAFF0028E1D1F3E7080001F0EEFF41
:106620000028DAD003780320A342D7D12900300014
:1066300004F02EFFD2E7C046FEFF00009866FF1F61
:10664000FFFF00009566FF1F9466FF1FF7B504006B
:10665000808801F0D3FF0025A84203D00578A088E8
:1066600002F008F81C4E3378002B1FD0AB421DD12E
:106670001A4B28001978FFF777FF002818D000235D
:106680003370A3790820A778A688019304F0C0FF8F
:10669000011E0DD0D0230370CA3B8370019B47704D
:1066A00086808371280005F0DBF801E0002DE8D139
:1066B000A0880B4B8200D358002B01D0FFF762FF5C
:1066C0001721A088FFF768FDA08801F027FDA088AA
:1066D00001F0FEFDF7BDC0469566FF1F9466FF1FE3
:1066E0009C66FF1FF0B587B01D000CAB1B88070030
:1066F00001930DAB1B88142002930EAB1B88160070
:1067000003930FAB1B880091049310AB1B88059378
:1067100004F07EFF041E1AD0D0230370CB3B4770D9
:106720008370C670062229000430002D11D004F0B9
:10673000CFFE019B21006381029B0098A381039BF4
:10674000E381049B2382059BA37405F089F807B0BD
:10675000F0BD04F03DFEECE7F7B5009308AB1B88F5
:1067600007000C200D001600019304F051FF041ED9
:1067700013D0280001F042FF00280FD00078D0236A
:106780002370C93BA370009B21002381019B67708C
:10679000A580E680638105F063F8F7BD014B1878AA
:1067A000EDE7C0460045FF1F13B504006489038967
:1067B000C2888188C0780094FFF7CEFF13BD000027
:1067C00010B5044C2068002803D004F069FE0023B3
:1067D000236010BDA066FF1FA122F0B58188920042
:1067E0004A43384B384F1B6804009B189D22920087
:1067F0009B18827989B01A603B68002B5FD01D78A6
:10680000324B1B68002B04D05B68002B01D00020AA
:106810009847260008363100E079FFF7B7FD237D61
:10682000E0710200E0780493638A29000393238ACD
:106830000293E3890193A38800933300FFF752FF8B
:10684000E378002B0BD1E289A379A188029201960B
:10685000E27928000092012201F0DAFEE0703B6844
:10686000002B20D0FFF7ACFF194D287800281AD054
:10687000184B1978FFF778FE002814D02B78E678AB
:1068800008200793A78804F0C3FE011E09D0D02377
:106890000370CA3B4670837087808671079804F046
:1068A000DFFF00232B701721A088FFF775FCA0885D
:1068B00001F034FCA08801F00BFD09B0F0BD064BDF
:1068C0009DE7C0463409FF1FA066FF1FB466FF1F87
:1068D0009566FF1F9466FF1F0045FF1FF8B5070070
:1068E00008000E0001F08AFE041E18D02620FFF7D3
:1068F0008DFC051E00D12578062004F089FE041EBB
:106900000DD00021062204F063FDD0232370C23B8A
:1069100021006770A370A680E8B204F0A1FFF8BD63
:10692000F0B585B001930AAB1B78070002930BAB5F
:106930001B7808000D000092039301F05FFE061E15
:1069400022D0102004F064FE041E1DD0102200216D
:1069500004F03EFD2620FFF759FC002800D13078D6
:10696000D0232370C13BA370009B21002372019BA5
:1069700067706372029BA580A372039BC0B2E3722F
:106980000C9BE36004F06CFF05B0F0BDF7B50D00A3
:10699000019001F033FE071E20D00E2004F038FED7
:1069A000041E1BD02620FFF731FC061E00D13E78C6
:1069B000D0232380C53B0622A370F91DE01C04F000
:1069C00087FD019B2A0063810123DD401A401D40A1
:1069D000210022736573F0B204F042FFF7BD00009E
:1069E000F0B585B0029010000D0017000A9E0393C9
:1069F00001F004FE041E31D0029B002B2ED1039B1C
:106A000002795B0724D5122313430422002E08D1F8
:106A10000B99002905D10C99002902D10D99002963
:106A20001AD01A430D9B2271002B00D0C9E0002E12
:106A300000D1CFE0002D00D0CCE0606A002801D06A
:106A400004F02EFD1C21300004F042FC606205E0E1
:106A500002239A430E33D7E793432371654BBA0061
:106A6000D458002C00D1AAE0002E10D0236A002BAD
:106A700003D11C2004F01CFD20625E4BBA00D358E9
:106A8000186A002803D01C22310004F021FD0C9B61
:106A9000002B12D0574CBB001D596B6A002B03D141
:106AA000162004F005FD6862BB00E358586A002810
:106AB00003D016220C9904F00BFD0D9B002B11D076
:106AC0004C4DBC006659B36A002B03D1142004F06E
:106AD000EFFCB0622B59986A002803D014220D995C
:106AE00004F0F6FC380001F089FD051E67D0414B2B
:106AF000BA00D358002B62D01A6A3420002A00D181
:106B00001C389A6A002A01D0143080B20B9A002AED
:106B100001D01C3080B25B6A002B01D0163080B2ED
:106B200004F076FD041E4AD01822002104F050FC27
:106B30002620FFF76BFB0190002801D12B780193F1
:106B4000D0232370029B200063700A23294EA37078
:106B5000039BBD00A371AB59A780196A18300029A7
:106B600005D01C22A06004F0B3FC2000343073591F
:106B7000996A002907D0030014221433E0600293BD
:106B800004F0A6FC02980B9B002B08D003001C22EB
:106B90001C330B992061029304F09AFC02987359FC
:106BA000596A002903D01622606104F091FC6B46FB
:106BB0002100187904F054FE3800FFF7E3FC05B01B
:106BC000F0BD10220D9B0D991B69A018236204F0E3
:106BD0007FFC2CE70B9B002B00D13FE7012D00D061
:106BE0003CE7606A002801D004F05AFC1C210B9895
:106BF0002AE7C0469C66FF1F10B5044C2068002899
:106C000003D004F04DFC0023236010BD9066FF1FED
:106C10000B4B07B51A68002A01D100200EBD69464A
:106C2000531C012012780731FFF772FC0028F4D0C2
:106C300002780123100018401A42EED0EEE7C04659
:106C4000AC66FF1FF0B51F4F01203B6887B0002BDB
:106C500025D09B78059300F0B3FB002821D00A20B3
:106C6000FFF7D4FA04000B20FFF7D0FA164B05000B
:106C70001E78731E9E413B68F6B2191DD878FFF747
:106C800057FB3B682900DA7A043303929A7901931F
:106C90000292009033002000059A04F089FC07B0AE
:106CA000F0BDFFF7B5FF002805D00620FFF7AEFACC
:106CB00004000720D8E70820FFF7A8FA04000920FD
:106CC000D2E7C0469066FF1F8C66FF1F70B50A4E64
:106CD000040033780D00FF2B0DD0042004F098FC45
:106CE000011E08D0D0230370CE3B45708370C47062
:106CF000307804F0B5FD70BD1045FF1F70B504007D
:106D000006200D0004F084FC011E0AD0D02303707D
:106D1000CD3B8370054B44701B688580187804F068
:106D20009FFD002C01D0FFF767FF70BD9066FF1F2D
:106D3000F8B5264F06003B680D001124002B05D145
:106D40000522234B1B78134202D112242000F8BDE8
:106D5000204A10241268002AF8D01278002AF5D0B0
:106D6000DB0719D52B789A1E012A1AD80C2004F0BB
:106D70009FFB132438600028E8D000230A224370C8
:106D800029000670023004F0A3FBFFF75BFF041E2E
:106D90000AD0FFF731FFD9E700F012FB0028E1D15C
:106DA000E4E7002BE2D0D0E70B4B1B78032BCDD1CF
:106DB0001D20FFF72BFA094B18800028C6D0084B7E
:106DC00004211878074A04F0EBFBBFE79066FF1F29
:106DD0008D66FF1FAC66FF1F8C66FF1F8A66FF1F54
:106DE000B866FF1F60EA0000F7B50193194B140065
:106DF0001A78052306000F0012201A4221D001291B
:106E000020D1154B1D68002D1BD002201F2C18D837
:106E1000002C02D0019B002B13D0104B1F221E70A0
:106E20006E1C0021300004F0D3FA019922003000DA
:106E300004F04EFB310020002C70002F06D004F02F
:106E40007FFBFEBD064B12201D68DCE704F098FBBB
:106E5000F7E7C0468D66FF1FAC66FF1F1045FF1F9A
:106E6000A866FF1FF8B50F4E12243368002B17D009
:106E70001B780F3C834213D100250B4F0221387839
:106E800004F05EFD094B042138781D8004F058FDA4
:106E9000074B28001D8033685C7004F061FB040020
:106EA0002000F8BD9066FF1FB866FF1FA466FF1F95
:106EB0008A66FF1F70B5012823D11B4C2388002B45
:106EC00003D01A4A1578002D07D0194B1B68002BE8
:106ED00002D01878FFF7C6FF70BD3B2B02D93C3BB0
:106EE0002380F9E7134E0221307804F029FDFA22BD
:106EF0002388920002215A43307804F019FB258040
:106F0000EAE70B4B1B68002BE6D00B4B1B785B07AB
:106F1000E2D5084B0221187804F012FD0022024B42
:106F20001A80FFF769FED7E7A466FF1F8866FF1F78
:106F30009066FF1FB866FF1F8D66FF1FF8B51E4DD8
:106F40002868002803D004F0ABFA00232B601B4E06
:106F50003068002803D004F0A3FA00233360184FF0
:106F600005243B7818002040234221D0154800F02A
:106F70002BFA3B78234213D0202004F099FA2860A2
:106F8000002813D02022002104F022FA202004F04F
:106F90008FFA041E306005D02022002104F018FA78
:106FA000002004E0286804F07BFA2C601320F8BD70
:106FB00000F00AFAF4E7C046AC66FF1FA866FF1FA0
:106FC0008D66FF1F0445FF1F10B50A4C23681A1E6B
:106FD0000ED0002808D10130587004F0C1FA002802
:106FE00005D02368002B02D00021FFF787FE012285
:106FF000100010BD9066FF1FF7B5274E05003368DF
:107000000191181E21D05C78244F012C30D1FFF75C
:10701000FFFD002825D02000FFF7F8F804004128E4
:1070200014D91F4B022118781E4A04F0B9FA1E4BDE
:107030003C3C1C80022233685A703B78002B14D1F0
:1070400028000199FFF75AFE0120FEBDFA229200A6
:107050004243002AEED0124B0221187804F068FA5D
:10706000E8E7FFF7D3F80200F3E700233B70EBE714
:107070003B78002BE8D1032004F0CAFA011E08D0A7
:10708000D0230370CC3B457083703368187804F0CC
:10709000E7FBFFF7B1FDD7E79066FF1F8866FF1F8C
:1070A000B866FF1F60EA0000A466FF1F10B517490D
:1070B000838802008B4220D011D815498B4217D00B
:1070C000144900205B1899B2012907D892681178F9
:1070D0005A425341D8B2FFF7F9FD012010BD0E4AC4
:1070E00000209B1807229BB29A424041C0B2F5E7AC
:1070F00083681878FFF768FFF0E7836899785A7813
:10710000090218781143FFF777FFE7E70A2000002C
:1071100006200000F8DFFFFFAFDFFFFF014B187014
:107120007047C0461145FF1F10B5064C207001F096
:1071300041FA207804F0E4F90521207800F062FD9E
:1071400010BDC046B866FF1F0BB273B50D00002B13
:1071500000DBC4E0884B187804F022FB041E0ED03C
:107160000378912B0FD0A22B00D1A1E0834B18788C
:10717000FF2852D0210004F073FB00284DD180205D
:107180000002684076BD43780F2B76D013D8052BCC
:1071900070D00E2BEAD18088794B98422BD8794B4E
:1071A00098421BD8784B9842E0D1A3681878591CB4
:1071B000FFF774F838E03E2BD8D18378032B74D0D6
:1071C0006CD8012B6ED0022BD0D1704B1B68002BDA
:1071D00023D05B68002B20D098471EE06C4BC01872
:1071E0000C28C3D804F044F91DC2C2150BC20B0B06
:1071F0000B3223C23C00674BC0180728B6D8664B39
:107200001B68002B09D01B68002B06D02000984774
:107210000AE0A3681878FFF7C7F8200004F0F0F838
:10722000ADE7A068FFF762F800289FD0F5E7A368F4
:107230001B78002BF1D0554B1B68002BEDD01B6841
:10724000002BEAD0210055489847EDE74F4B1B68CB
:10725000002BE2D01B68002BDFD021005048F3E761
:10726000504B1B68002BD8D05B68002BD5D0210079
:107270004348E9E7FFF7EAF9CFE780884A4B9842AD
:1072800003D04A4B984200D070E7464B1B68002B56
:10729000C3D05B68002BC0D02100D5E7153B012B84
:1072A000BBD963E7FFF798FAB7E7FFF77DFAB4E7D2
:1072B0003F4B1B78042B07D100236A4613800179CA
:1072C000408800F0C5FCA8E7364B1B68002BA4D013
:1072D0005B68002BA1D00100364898479DE7012448
:1072E00021420AD0294B1B68002B04D05B68002B7D
:1072F00001D000209847012043E78B070AD5264B91
:107300001B68002B04D05B68002B01D0200098473D
:10731000022036E70421280008400D4200D131E761
:10732000254E3388002B21D0013B9BB23380002BAC
:107330001AD1FFF7DBF800280AD0204B1C70164B3F
:107340001B68002B04D05B68002B01D020009847FD
:10735000FFF7C6F8694601F001FD6846FEF7FEFF3B
:107360001D20FEF753FF308004200AE7024B1878F7
:1073700004F0E6FAF8E7C046B866FF1F1145FF1FA4
:107380000E2000000120000009100000B066FF1F61
:10739000FEDFFFFFAFDFFFFFB466FF1F0C20000022
:1073A0000B2000009866FF1F0D2000001320000036
:1073B0008D66FF1FFFFF00008A66FF1F8866FF1FA4
:1073C00010B501F09BF910BD014B18607047C04625
:1073D000B466FF1F0B880020162B01D8172304204A
:1073E000014A13807047C0466266FF1F0020704745
:1073F000074A03001188814207D0918800209942F2
:1074000002D101308000101870470020FAE7C04612
:10741000C066FF1FF0B58F7806000D00C7B01E2FA5
:1074200015D1FFF7E5FF051E03D10024200047B06A
:10743000F0BD00223B003100C078009200F0B2FBAA
:107440000400A81C00F0D3FBFF23EB70EEE7264BF3
:10745000062403931B78FF2BE8D0182FE6D87B086F
:10746000224A013BDB0002929A589446002ADDD062
:10747000029AD3185B68002BD8D00878002802D174
:107480004B78012B02D10624122FCFD107AFAB8846
:10749000697800976446AA68A047041EC6D1AB78F5
:1074A000029A5B08013BDB00D318390030005B68AF
:1074B0009847041E0BD1AB78042BB6D0039A310049
:1074C00010782200009700F06DFB0400AEE76A78A8
:1074D000002AABD1AA7805A93B88087130000A7050
:1074E0004B80FEF747FBA0E71445FF1F6CBB001164
:1074F0001D4B37B5050098420BD000290AD1FFF784
:1075000077FF002805D11948FFF772FF002800D047
:10751000058037BD01291AD1FFF76AFF041EF8D094
:1075200001235B420380A378FF2BF2D0FE2B07D010
:107530000023E0781422009329001E3300F032FB70
:10754000A01C00F054FB01235B426380E1E70229A9
:10755000DFD1013901F0BEF80028DAD12800FFF7A9
:1075600047FF041EDFD1D4E7FEFF0000FFFF00004D
:10757000022210B5074B52421A80074801325A8046
:107580009A80DA8000F07EFA044801F025F80020A5
:1075900010BDC046C066FF1F15740011F1740011C4
:1075A0000388F7B50400002B02D102252800FEBD98
:1075B00042680221137825485268FEF7A5FD00288D
:1075C0002ED0234F01253A88002AEFD0802321882E
:1075D0005B0201259B1A9942E8DC0C2003F068FF4E
:1075E000061E31D03B8822889C4600231800019556
:1075F00061469DB2491989B2AA421BD8002801D020
:1076000062443A8000233000082208C0210003F0C1
:107610005FFF104A1368002B13D100251660C5E7E1
:107620006268022113780C485268FEF76DFD00284D
:10763000C7D1BAE760681D01401941810133019843
:10764000D6E71A001B68E6E71325AFE7DABB00119F
:107650001245FF1FBC66FF1FD8BB0011014B1870FD
:107660007047C0461445FF1F14230A0010B51A4086
:10767000194204D00122102101F048F810BD4B0638
:10768000F9D4012088434000F8E710B514008B06B8
:1076900004D50122102101F039F810BD08230A0099
:1076A0001A40194202D14BB2002B0FDA102101F01F
:1076B0002DF8002808D02300F9331B78002BECD0DC
:1076C000F8342378012BE8D10020E6E7032089076E
:1076D000FAD4E2E7F0B51F00184B85B01C680190A2
:1076E00002910392002C27D1200005B0F0BDA568BF
:1076F0003301ED186B89019A934211D3029A934298
:107700000ED8002F04D10A9B002B10D12C00EBE7E0
:107710003B002978039A6868FEF7F6FC0028F2D14E
:107720000136B6B2A388B342E1D82468DAE7A36889
:107730000A9A5B891380E9E70026F3E7BC66FF1F1E
:1077400037B50C000A8849880123914217D3002AD3
:1077500015D0651D23792A0002210A48FEF7D4FCC2
:10776000102300280BD023796188208800242A0068
:107770000094FFF7AFFF0A23A04200D023001800B7
:107780003EBDC046DABB001113B50A00088849881F
:10779000012388420BD8002809D000241379053230
:1077A0000094FFF797FF0A23A04200D0230018009F
:1077B00016BD13B50A0008884988012388420BD8F2
:1077C000002809D00024137905320094FFF782FFC6
:1077D0000A23A04200D02300180016BDF0B58BB0DC
:1077E00003904A8808880E000123824255D300285E
:1077F00053D00023012704AC2370002271881300AA
:107800000092FFF767FF051E3ED02078002835D193
:107810002B78022B18D167706A8983000130E31836
:1078200080005A8069680222201803F051FE2378F4
:107830000133DBB22370042B19D93B006889013076
:1078400080B2002BD9D01FE002236370122358436B
:107850006A89231804305A8069681022201803F0BE
:1078600037FE23780133DBB22370002BE5D10C4ABD
:107870006B899B185A425341DBB2DFE76378012BD7
:10788000E4D12B78022BC7D022780A23002A04D017
:1078900021000398FEF798F9002318000BB0F0BD03
:1078A0000100FFFF0F4BF0B504001868002816D048
:1078B00083685D89A54207D88288AE18B44203DA8E
:1078C00012019A18934201D10068EFE71E005F8908
:1078D0001036A74204D1002900D00D801800F0BD59
:1078E0003300EFE7BC66FF1F70B505000C00088889
:1078F0000021FFF7D7FF03000120002B04D0220056
:107900002800197AFFF7C1FE70BDF7B50C000025FD
:1079100001902300F6331B78AB4201D800200AE027
:107920006B00E65A00213000E718FFF7BBFF002884
:1079300002D126800130FEBD017A0198FFF794FE46
:10794000002802D03B882380F5E70135EDB2E0E75F
:1079500010B5040008880021FFF7A4FF03000120F0
:10796000002B03D02000197AFFF77EFE10BD000027
:10797000054B1B68002B01D1180004E09A6852895E
:107980008242F6D198887047BC66FF1FF0B50E277B
:10799000002687B0039302ABFF183E8005001F4B03
:1079A00040891400984207D02B78013000976A680C
:1079B00080B2FFF78FFE060002212B7818486A6814
:1079C000FEF7A2FB00280FD06C892000FFF7D0FF44
:1079D000002802D0013C0419A4B2039B002B00D064
:1079E0001C80300007B0F0BD02212B780D486A687A
:1079F000FEF78AFB0028E7D102212B780A486A6843
:107A0000FEF782FB002807D0002EDED03B88A34281
:107A1000DBD17489013CDFE76C89DEE7FFFF000002
:107A2000DABB0011D8BB0011D6BB001110B50C0099
:107A3000FFF7DEFC03000220002B0AD0002C00D050
:107A400023609B781720FE2B03D00138FF2B00D139
:107A5000002010BD73B50D0001A904001600FFF74A
:107A6000E5FF172805D0002E04D129002000FEF7DD
:107A700027F976BD01221021200000F047FE0028E2
:107A8000F3D0F6E7014B18607047C046CC66FF1F85
:107A900037B56B469D1D010004000222280003F04B
:107AA00067FD2B88B02B0ED12379122B09D123002F
:107AB000FF339B78012B06D10121608800F0E0F8AC
:107AC00001E01B2BF8D037BD10B5054B0421187011
:107AD00000F098F8FFF74CFDFEF770FB10BDC046B4
:107AE000D066FF1F0020F0B50BB20F0087B08342B5
:107AF00034DA274B187803F053FE051E2BD0037899
:107B0000A02B25D103AE3100FEF7E4F8041E0BD103
:107B1000B378DB0724D51F4B06341B68002B03D03A
:107B20003100688898470400A868002801D003F055
:107B30000FFF002C08D1184A039B1340174A9342A9
:107B400006D0B3781B2B03D00121688800F098F889
:107B5000280003F055FC80200002784007B0F0BDFB
:107B60000F4B1B68002B10D0310068889847041E0B
:107B7000DAD07378002BD7D1B27801A90A704B8084
:107B80000C716888FDF7F6FFCEE70624F1E7C046E2
:107B9000D066FF1FC866FF1F00FFFF000001120034
:107BA000CC66FF1FF7B50190822040000D00170042
:107BB0001E0003F02DFD04001320002C12D0B02372
:107BC00020002370089BFC226770658026710830B6
:107BD000002B08D0190003F07BFC2100019803F072
:107BE0003FFE0020FEBD089903F0F2FBF5E710B55B
:107BF000041E06D00078FD2803D803F019FDFF23EA
:107C0000237010BD0A1F93B210B504000220032B8D
:107C100005D882400020024BD1529B189C7010BDA9
:107C2000F066FF1F0B8870B5043B04000D000220B6
:107C3000032B0BD80121200000F04CFD0300142081
:107C4000002B03D02900200000F0DEFB70BD0000F7
:107C500007B51300034A00920A00012100F02CFC32
:107C60000EBDC0468D7E001107B501920322009221
:107C7000024B0A00122100F049FC0EBD0B7F0011DF
:107C800007B56B4601AA11800449D88008780633ED
:107C9000012802D1190003F01BFD07BDD166FF1FAB
:107CA0000C4B10B518700023FF210B4A1380138171
:107CB00093819380094A5380137051729381937218
:107CC000D174D3821375517703F0A2FD00F0FCF953
:107CD00010BDC0460067FF1FF066FF1FD266FF1F82
:107CE000F0B58DB06B46002003910C229B5E834261
:107CF00000DBB0E05D4B187803F052FD051E00D1AB
:107D0000A4E00378902B00D09DE006AF01004688E8
:107D1000380000F013FA79680400002900D19CE0D3
:107D20003B88052B6ED13B89032B1CD905AC200069
:107D300000F0A2F86288172A61D83989131D994288
:107D400031D17968237804310291D90738D5607828
:107D500000F08EF9071E06D0002303712378012B53
:107D600008D0132B23D0A868002800D178E003F0B6
:107D7000EFFD75E06288029909A800F0A6F802906C
:107D8000380000F08BF909AA2378387A0192002292
:107D900031000092029A00F012F9380000F064F904
:107DA000029B002BDFD0300000F080F9DBE7037886
:107DB000032BD8D16288029909A800F0D6F8DEE733
:107DC000122B13D1029909A800F0B5F8021EEAD1CE
:107DD00027498B88002BC6D0887909A9237801917F
:107DE00061780091310000F0EAF8BCE7002302AAB4
:107DF00093833000617809AAFFF72AFFB3E71D4B90
:107E00000993F6E7042B02D09A1F012AABD8184A2F
:107E1000043B9B00995A0029A5D0D21890783100D4
:107E20003A0000F0AEF800289DD13B88042B03D027
:107E300001213000FFF724FF012C04D1A86800289D
:107E400001D003F085FD280003F0DAFA8020039BBF
:107E50000002434018000DB0F0BD012800D182E7B8
:107E600001213000FFF70CFFEDE7C0460067FF1F60
:107E7000F066FF1F010017000B7803704B7843700A
:107E8000CB788A781B021343438070470A8803002B
:107E900002700A88120A42700A88012A06D14A88AA
:107EA00082704A88120AC2700420704702208242FF
:107EB000FBD14A8804309A704A88120ADA708A889C
:107EC0001A718A88120A5A71EFE710B5040001206E
:107ED00082420CD94B780A781B02134323808342D9
:107EE00006D1CB788A781B0213436380002010BD33
:107EF000022BFBD1CB788A781B02134363804B792A
:107F00000A791B021343A380F0E70B8803700B88E8
:107F10001B0A43704B8883704B881B0AC3708B8885
:107F200003718B881B0A4371CB888371CB881B0A32
:107F3000C3710820704703000120082A14D14A7831
:107F40000878120202431A80CA7888781202024323
:107F50005A804A790879120202439A80CA7988794C
:107F6000120202430020DA80704710B5040001209D
:107F7000022A05D100204B780A781B021343238084
:107F800010BDF8B5060010200F00150003F040FBEF
:107F900004000120002C0ED0A0230C2229002380F5
:107FA0006780201D002D07D003F092FA21003000D9
:107FB00003F056FC0020F8BD03F00AFAF6E7F7B527
:107FC0001E00009008AB142017001D78019103F0EB
:107FD0001FFB041E12D0A2230370019B4770438035
:107FE000099B057146710C220830002B07D019003F
:107FF00003F06EFA2100009803F032FCF7BD0999F6
:1080000003F0E6F9F6E737B5041E0FD04388002BDE
:108010000CD00025C1881323007A17220195009502
:10802000FFF7CDFFFF2365806372257037BD000029
:1080300010B50C4904004A88002A09D08B89002B0E
:1080400005D00020CB8A0222834201D010BD01223C
:1080500013000A20434300204032C854C81842800D
:108060000472F3E7D266FF1F00234380037070475A
:10807000094B00211A0010B55C88002C06D01C7931
:10808000844203D10A234B43D01810BD01310A3377
:108090000329F1D10020F8E7D266FF1F10B50400D4
:1080A000407A03F0C5FAFF23637210BD70470430B5
:1080B00010B580B203F06CFA002803D004214942C5
:1080C00003F016F910BD000070B50025104CA06833
:1080D0002580A581A580A84202D003F039FCA560C7
:1080E00000250C4C0C4B606D1D80230058331D7017
:1080F000A84202D003F02CFC6565002560680028CA
:1081000001D003F025FC013508340A2DF6D170BDED
:108110009867FF1F3C67FF1F8C67FF1F70B5041E29
:1081200009D1054D2880A881A880A868002802D020
:1081300003F00EFCAC6070BD9867FF1FF0B54B8874
:1081400085B00193002343600A7905000F00022ADD
:1081500000D07BE0CA88032A17D98B685E7819782B
:108160003602DC78D8790E4399781B7A24021B02F8
:108170000C43034353495BBA0B80331D93421ED11A
:10818000042C04D0631F022B0ED9012015E0019AA4
:108190004D4B1201D35A002B06D00198FFF7BEFFBA
:1081A0004A4A1369013313610421B8682E812C8077
:1081B000494203F09DF86860002005B0F0BD434DD2
:1081C000042C06D0631F022B0FD9EB680133EB6040
:1081D000DBE7019A3C4B1201D35A002B05D00198E2
:1081E000FFF79CFF2B6901332B61374B3000029363
:1081F000019B029A1B010193002301998C468B522B
:10820000130063449C8003939E81FFF750FF039B00
:10821000041E986016D00421B868494203F068F83B
:10822000FA880100043A200003F052F90199029AF9
:10823000FB888A5A043B9B18029A8B522B680133A5
:108240002B60A2E7AB690133AB619EE71E4B029343
:10825000019B1E01029BF35A002B2DD002998C1911
:10826000A068002828D0012A26D1FA889B189BB242
:108270007352A189994217D39B1AC018B96803F0A9
:1082800027F9029BA289F35A934200D07DE700228E
:108290002B81A3882B80A3686B60029BF2520B4A50
:1082A00053680133536070E7084A93680133936061
:1082B0000198FFF733FF68E7044A536901335361BC
:1082C000F6E7C0460267FF1F9867FF1F0867FF1F9A
:1082D00070B5051E15D10B4C0B4B1880230058337D
:1082E0001870606D002802D003F032FB6565250030
:1082F00050356068002801D003F02AFB0834AC42F6
:10830000F7D170BD3C67FF1F8C67FF1FF0B51700EA
:10831000A12285B0920001934243394B06001B68AD
:108320000C009B18D933FF331D78FDF741FF043053
:10833000854204DD3000FDF73BFF0430C5B2BD428D
:1083400007D33A0000213000019B03F081F905B00A
:10835000F0BD2900380003F08BFA2300C6B2503379
:108360001E700393019B29006365380002F0D0FF63
:10837000CBB20293002B02D0039B01361E70002665
:108380002300503303931B78B34204D8606D002858
:1083900031D10020DBE7029A2800002A04D0013BFB
:1083A0001000B34200D02800F700E719387002F03F
:1083B000D7FF786000280ED03A78019903F088F84A
:1083C000019A3B780136D3180E4A0193D369F6B26D
:1083D0000133D361D4E7039B18706065A74205D1D0
:1083E000084A1320D36A0133D362B0E7606803F010
:1083F000AFFA0834F2E703F0ABFA00236365C8E78D
:108400003409FF1F0867FF1FF7B50D00070004219F
:10841000686802F06DFF2B89040003702B891B0A2A
:1084200043702B8883702B881B0AC3702E8902250A
:108430000436F6B2FB2E15D81B4B9F4214D10C20EC
:1084400003F0E6F81135011E0CD0902303708E3B2B
:108450000371043B4380154B8460C680187803F099
:10846000FFF900252800FEBD5C237B43104AD3188A
:108470000093583301931B78002B0FD10300320077
:1084800038000099FFF742FF019B05001B78002B85
:10849000E8D13800009902F073FFE3E7054A0725A9
:1084A000536A01335362DDE7FEFF00000067FF1FE0
:1084B0003C67FF1F0867FF1FF0B587B000901720CB
:1084C0000F0016000193FFF7F2FD1325041E19D0CB
:1084D0000C98031E02D00199201D9847030AE370EF
:1084E000052302AAA070043090812770009866705E
:1084F00003A993800494FFF787FF051E02D0200094
:1085000003F026FA280007B0F0BD0000F0B587B0F0
:108510001F000CAB1B780391059301210DAB0600E6
:108520001C78049200F0D6F81425002821D02000F1
:10853000FFF77EFD0135041E1BD01149059B0A780B
:1085400003700132D2B2131EC68001D101231A007A
:108550000B7022713000049B03990097FFF7ACFF6A
:10856000051E09D1230021000648074A093303F0FC
:108570009FF9280007B0F0BD002363802370F8E75F
:108580000467FF1F0780001130750000F8B5050073
:108590000E00064C064F2368002B02D03100280045
:1085A00098470434BC42F6D1F8BDC046A867FF1F07
:1085B000BC67FF1F0123064A5B42538000231371EF
:1085C0005362044A136053609360D3601361704731
:1085D000BC67FF1FA867FF1F0200002310B50649F4
:1085E0009C000859002801D1625010BD0133052BB1
:1085F000F6D11320F9E7C046A867FF1F034A538846
:10860000181A43425841404210407047BC67FF1F50
:10861000F0B585B002930AAB1F780CAB1B880090B5
:1086200008000E0001920393FFF7E8FF05001120F8
:10863000002D1BD10E48FFF7E1FF04001520002C90
:1086400014D006220B99A771E01D02F041FF019B97
:1086500030002371029B29006371009B66802370A8
:10866000039B6562E381FFF791FF280005B0F0BD31
:10867000FFFF000010B5FFF7C1FF04000220002C2F
:1086800012D060880121FFF781FF606A002801D0C5
:1086900002F006FF28220021200002F099FE0123AB
:1086A00000205B426380207110BD000030B5074A96
:1086B000074C5588010013780020A54204D05B1AAE
:1086C00059424B415842104030BDC046BC67FF1F65
:1086D000FFFF0000084A10B501230C00904208D0AB
:1086E000FFF78CFF031E04D0037923405A1E9341E9
:1086F000DBB2180010BDC046FEFF0000024B187927
:10870000431E9841C0B27047BC67FF1F70B504009C
:108710000D001600FFF772FF002804D10D4B9C429C
:1087200000D0143070BD416A03790520002907D0BC
:1087300012221A40102A02D10520002EF2D10F2059
:10874000DB06EFD5897E0C20A94289414942494286
:108750000840E7E7FEFF0000030010B5002800D145
:1087600010BD0348034A41889142F9D09847F7E782
:10877000BC67FF1FFFFF0000002330B5C45CCD5C69
:108780006C40D4540133102BF8D130BD0F2300229C
:1087900010B5C45C64002243CA54C25CD209013BD8
:1087A000F7D210BD0200010010B52032103103F0E5
:1087B0001FF810BDF0B58BB0039010200593170083
:1087C000049102F075FE0090102002F071FE009BF3
:1087D00013240190002B05D000280CD113240098FD
:1087E00002F05EFE019B002B02D0180002F058FE42
:1087F00020000BB0F0BD102002F05AFE0600102041
:1088000002F056FE13240500002E00D1AEE0002831
:1088100019D01022002102F0DBFD3200290003985C
:1088200002F0E6FF041E0ED133787F2B51D83000C2
:108830000099FFF7ABFF009B1B787F2B53D8019962
:108840000098FFF7A3FF300002F02AFE002D02D0AF
:10885000280002F025FE002CC1D1102002F028FED5
:108860000600102002F024FE0290002E7CD000288A
:1088700078D03A000F3223000125121105D00F33B2
:108880003B4015B25A4253411BB26A1E1201002BE3
:1088900033D0049BD2B298180099029AFFF76CFF6C
:1088A000013D10220021300002F092FDADB2049F84
:1088B0002D017D19AF4242D0002C33D0300002F0A0
:1088C000EFFD029B002B00D189E7180002F0E8FDC4
:1088D00085E729003000FFF759FF28002549009A55
:1088E000FFF74AFFA7E729000098FFF74FFF28008E
:1088F0002049019AFFF740FFA5E70F210F40049997
:108900008A18D9B28F4208D9D15C06A8195401330C
:10891000102BF6D1029A0199C0E7791A48424141D9
:10892000C901F2E73900300006AAFFF725FF32003F
:10893000039806A902F05CFF10370400BAE7002C88
:10894000BCD13000029906AAFFF716FF320006A933
:10895000039802F04DFF082204003100059802F050
:10896000B7FDABE71324A9E71324AAE7002800D03A
:108970006EE733E7E0BB0011F0B58BB00F001600D7
:108980000225009000283FD0002A3DD00B1DDBB20D
:108990001800029302F08CFD1135041E34D0FDF74F
:1089A00047FD05003A000099201D02F061FEEBB280
:1089B0000393E3702B0CDBB22F0A00936370FFB2BA
:1089C0002B0E2370A7700193FDF72CFD10220100E0
:1089D00006A802F04DFE2100029A04AB06A8FFF79C
:1089E000E9FE051E0DD1039B08223370009B04A9EC
:1089F000B370019B7770F370301D02F039FEFDF704
:108A00001DFD200002F04CFD28000BB0F0BDF0B5BC
:108A10008FB00D00149E039004920593002A03D199
:108A2000022420000FB0F0BD002EF9D00398FFF70C
:108A3000E5FD1424071EF4D07278337812021A432D
:108A4000B3781B041343F27812061A43036A0192A7
:108A5000934201D30133E3D1002D03D03B790124AC
:108A60009B07DED50822002106A802F0B1FC059B79
:108A700013240433DBB21800029302F019FD051E23
:108A8000CFD0059A0499043002F0F2FD042231009F
:108A9000280002F0EDFD3900102210310AA802F082
:108AA000E7FD2900029A06AB0AA8FFF783FE041E21
:108AB0000FD1082206A908A802F0DAFD0822311D0C
:108AC00008A802F025FD012807D101990398FDF7B8
:108AD000C9FC280002F0E4FCA3E70124F9E7000048
:108AE00070B51C4C05002368181E10D0002D14D141
:108AF0001A78002A0CD1981C083202F0E9FC02F026
:108B0000DFFC0135002808D123681D70012070BDED
:108B10000A331800082202F0DBFC2368002BF5D092
:108B2000122002F075FD061E0DD0C12321680370CE
:108B3000457002311022023002F0CAFC2368310075
:108B4000587802F08DFE206802F0AAFC0023236012
:108B5000DCE7C046E467FF1FF8B504002020FDF7FE
:108B600055FB0D4EA700BB590500002B0DD000286A
:108B70000BD0D878FF2809D108492A000C55F359A1
:108B800007480333611802F093FEF8BD290002F094
:108B90001FFD0028F0D1F8E70068FF1FE867FF1FFE
:108BA000B19D001170B5064D84006359002B05D0AE
:108BB000D87802F03DFDFF226359DA7070BDC046DF
:108BC0000068FF1F70B506008CB00C001500002176
:108BD0003022684602F0FCFB31001022684602F0A9
:108BE00047FD1D2021000322684402F041FD684634
:108BF000FFF7D8FD2D21040003222800694402F06C
:108C000037FD20000CB070BDF0B50700160097B01E
:108C100001931CAB1D7830221EAB00910AA80021E5
:108C20001C7802F0D5FB102239000AA802F020FDC2
:108C30001022002102A802F0CBFB0722310002A87B
:108C400002F016FD072202AB9818631E9C410199A1
:108C500002F00EFD02AB9C732B005A1E934102AA38
:108C6000D3730021102206A802F0B2FB06221D9940
:108C700007A802F0FDFC1A2002ABC01806221F99BB
:108C800002F0F6FC102200990EA802F0F1FC10226E
:108C900002AB0EA908781C78013A6040D2B2087085
:108CA00001330131002AF5D10AA8FFF77BFD10221C
:108CB00012A904000EA802F00BFC102206AB0EA9AC
:108CC00008781D78013A6840D2B20870013301314A
:108CD000002AF5D10AA8FFF765FD04431022209869
:108CE000E4B212A902F0C4FC200017B0F0BD70B5C8
:108CF0000E0014008CB00100102268461D0002F026
:108D0000B7FC3100082204A802F0B2FC21000822BE
:108D100006A802F0ADFC6846FFF744FD04001022EF
:108D2000280008A902F0A4FC20000CB070BDF8B522
:108D300006000D0000243719AC4200D3F8BD02F044
:108D4000A7FD030A3B70631CDBB201379D4203D9C8
:108D50000234F054E4B2EEE71C00EDE773B5060010
:108D60000C000225002819D0002917D0032101A8E2
:108D7000FFF7DDFF6B469A793F231A400133134317
:108D80006A463000937101A92200FFF71BFF051E00
:108D900004D10322E01C01A902F09AFB280076BD51
:108DA00003785807DA08C00FD20080009B071043F1
:108DB0009B0F1843C0B2704707230B40C908C90076
:108DC0000B4303707047000070B50400FFF7EAFE24
:108DD000134DA4006359002B21D0186A002801D03C
:108DE00002F05EFB2B59986E002801D002F058FB70
:108DF0002B59D86E002801D002F052FB2B59186F66
:108E0000002801D002F04CFB2B59586F002801D0EC
:108E100002F046FB285902F043FB00232B5170BDA2
:108E20000068FF1F0E4B8000C35870B50C00002B6C
:108E30000FD09D68002D0CD02B78201D0B706B7807
:108E40004B70A97CFFF7B8FF2B7E23726B69E36040
:108E500070BD10220021200002F0BAFAF8E7C046E7
:108E60000068FF1F014B18607047C046FC67FF1F7A
:108E7000074A03008000825810B5002A06D0D08827
:108E8000984203D1012901D1FFF79EFF10BDC046D2
:108E90000068FF1FF0B5264E95B087000B93BB59B5
:108EA0000500099112200A92002B31D0D888FFF7D3
:108EB000A5FB04001420002C2AD0280010A9FFF7DD
:108EC000B1FFBB591E781D6A002E23D00895FDF70F
:108ED000EFFA07000020FDF7F1FA0790A379E61DED
:108EE000069310AD0CA9089800F0E2FA0EA928002C
:108EF00000F0D7FA0B9B0A990493069B09980293FA
:108F0000079B0396019300970EAB0CAAFFF77CFE1C
:108F100015B0F0BDFDF7CCFA06903000FDF7CEFAA3
:108F2000E31DA779079310AB06000893DAE7C04664
:108F30000068FF1F30B50C4C85002A59030085B02E
:108F40000120002A0ED018006946FFF76BFF2B594D
:108F50001A78D888054B002A00D1054B6A460721AC
:108F600000F0D9FB05B030BD0068FF1FA3940011CD
:108F7000B194001130B5094C8500295985B01022F3
:108F80006846253102F0A4FA2A591121044BD088F1
:108F90006A4600F0C0FB05B030BDC0460068FF1F48
:108FA0004D95001130B5094C8500295985B0102226
:108FB0006846353102F08CFA2A591121044BD088C9
:108FC0006A4600F0A8FB05B030BDC0460068FF1F30
:108FD0008B950011F7B54D4F86001020F4590D0008
:108FE00002F066FAF3592062186A132200286CD046
:108FF000033A29009C6802F06BFAF3591A7801923F
:10900000002A58D11E6A227D317B944651400122AC
:10901000019F114201D167461740217D9143394399
:109020002175377B4F40BC4660460027800701D43E
:109030004F081740012102208F40227D82433A438E
:109040002275377B5740BC4660460027400701D455
:1090500097080F400420227DBF0082433A432275C7
:10906000627D002794466046727B42400A4201D1ED
:1090700067460F400121627D8A433A436275777BE0
:109080005740BC4660460027800701D457080F4070
:109090000220627D7F00824317436775767B002242
:1090A0007E40760701D4BA080A400426617D92000A
:1090B000B1430A4362756A78002A08D06278002AB0
:1090C00005D005220533DA7700221000FEBD042208
:1090D0002979114205D1A17C114202D10533033A0D
:1090E000F1E7019A21782C78002A02D10A002100A8
:1090F000140018220429E8D8042CE6D8052060437F
:10910000034A05331218525CDDE7C0460068FF1FB2
:10911000F0BB001110B50A001121024B00F0FBFA60
:1091200010BDC046E79500110B0030B587B001AD0A
:109130002B806B4604001100981D082202F0C8F92C
:109140002A000B212000024B00F0E5FA07B030BDE9
:109150000F96001110B50A001121024B00F0DBFA46
:1091600010BDC0466396001113B50B0011006A468E
:1091700013706B4604000622581C02F0A9F96A46D7
:1091800008212000014B00F0C6FA13BD83960011A0
:1091900010B50A001121024B00F0BDFA10BDC04607
:1091A000D39600117FB505000B4BAA00D4580800D8
:1091B000002C0FD0666F237FE28821780396266FFC
:1091C0000296E66E0196A46E0094FDF709FC280055
:1091D000FFF7FAFD7FBDC0460068FF1F10B51721DD
:1091E000FFF7E0FF10BD000070B50A000D00064B50
:1091F0000221040000F08FFA060029782000FFF712
:10920000D1FF300070BDC046B395001170B586B077
:1092100000236A461370836804001D78681E0A28BC
:1092200059D801A902F0F4F8060633373B3F43470B
:109230004B4F5300180000F042F9062312284BD080
:1092400000281BD16088FFF7D9F90823002813D024
:109250004279002A47D1264B1A78072312070BD5EB
:10926000244B1A680723002A06D01668002E03D064
:10927000290001AAB04703006A4613706B461B78A9
:109280006088002B2AD1FFF767FC06B070BD18007C
:1092900000F06CF9D4E7180000F087F9D0E7180067
:1092A00000F093F9CCE7180000F0ADF9C8E718001A
:1092B00000F0C3F9C4E7180000F0F6F9C0E71800A1
:1092C00000F0F6F9BCE7180000F013FAB8E7180050
:1092D00000F013FAB4E707236A4613706946608802
:1092E000FFF782FFD1E70523012AC5D1024BB8E77A
:1092F0008D66FF1FF867FF1FFC67FF1FF8B52C4F37
:109300008600F35904000D00002B40D0DA88824219
:109310003DD15A78062A33D11A78002A2ED001205E
:1093200099681A6A097D014206D0157B054203D06F
:1093300007225A700120F8BD0220014204D0157B9B
:10934000054201D00922F4E70420014204D0127B37
:10935000024201D00B22ECE7164B1B68002BE9D030
:109360005B68002BE6D020009847BB5900215B7852
:10937000122BDFD12000FFF715FFDBE70E4BECE7E8
:10938000112A04D1002900D032252900F2E7002D4E
:1093900008D12000FFF732F9002803D0102302790A
:1093A0001343037121002800FDF798FAC2E7C04675
:1093B0000068FF1FF867FF1FFC67FF1F70B50E4EA8
:1093C0008500AB590400002B13D01B78002B11D162
:1093D0000A4B1B68002B04D05B68002B01D02000D7
:1093E000984773595B78122B03D100212000FFF7B7
:1093F000D9FE70BD024BECE70068FF1FFC67FF1F42
:10940000F867FF1F094B8000C3581020002B0CD0B9
:109410001A6A002A09D09B68002B06D0127A1B7E9C
:10942000101C9A4200D9181CC0B270470068FF1F78
:1094300070B503000D0014000220002A30D000296E
:109440002ED013700B78081D53704B789370FFF774
:10945000A7FCE070012002212B7A23716B7B034073
:1094600063716A7B0A401343042263716E7B16406A
:10947000334363716E7BF608F600334363712B7BD5
:109480000340A371287B014000200B43A371297B7B
:109490000A401343A3712A7BD208D2001343A3715D
:1094A00070BD10B50A0001000120FFF7C1FF10BD1B
:1094B00010B50A0001000220FFF7BAFF10BD70B519
:1094C00006000C000220002E30D000292ED0737828
:1094D000201D0B70B3784B70F178FFF76DFC012203
:1094E0003579257271794B10080013409340104074
:1094F0000343881010408000C9080343C9000B4390
:109500006373B1794B10080013409340104003433C
:10951000881002409200C9081343C9000B43212060
:109520002373FCF773FE854201D2122070BD222006
:10953000257AFCF76BFE8542F7D823781820042B98
:10954000F4D86378012BF1D80020EFE7030010B5C1
:109550000220002909D0002B07D00322481C0A70E2
:1095600019000D3201F0B4FF002010BD03000222EB
:10957000080010B5002B06D0002904D00E32591C6B
:1095800001F0A6FF0022100010BD030010B502205C
:10959000002909D0002B07D00422481C0A701900AA
:1095A0000C3201F095FF002010BD10B5FFF7DEFF73
:1095B00010BD03000220002906D0002B04D0052294
:1095C00000200A701B784B70704703000220002BAC
:1095D00008D0002906D05B7800200B70013B082BD7
:1095E00000D918307047030010B50220002909D0B7
:1095F000002B07D00622481C0A7019000A3201F01D
:1096000067FF002010BD10B5FFF7B0FF10BD0200CE
:109610000B00022010B500290ED0002A0CD0072123
:109620001970118859701188090A99701118082247
:10963000D81C01F04DFF002010BD03000A000220DD
:1096400010B5002B0CD000290AD09978587809025F
:1096500001431180901CD91C082201F039FF002021
:1096600010BD030010B50220002909D0002B07D03F
:109670000822481C0A701900921801F029FF0020E6
:1096800010BD02000B00022010B500290BD0002AEB
:1096900009D009211970117818185970511C062227
:1096A00001F016FF002010BD10B5FFF75FFF10BDE1
:1096B00002000B00022010B5002A09D0002907D0B3
:1096C0005178197011180622581C01F001FF002072
:1096D00010BD030010B50220002909D0002B07D0CF
:1096E0000A22481C0A701900063201F0F1FE00201F
:1096F00010BD10B5FFF73AFF10BD02000B000220AD
:1097000010B5002A06D0002904D018005178FFF7C0
:1097100053FB002010BDF0B585B017001E006A464F
:1097200006230500080091819380FEF7C0FC1324F6
:10973000011E02900CD03800B047041E05D128004D
:1097400001A9FEF76FFA041E02D0029802F000F998
:109750002800FFF701FA200005B0F0BDF0B50400C5
:109760008BB0019115000021102202A801F030FEFB
:10977000334EA700B85900283CD0C388A34239D142
:109780000378002B36D14278062A18D10200010056
:10979000553235310C3006ABFFF7A9FA002829D134
:1097A0002000FFF72FFE020006A902A801F090FE9C
:1097B000200002A901F01CFF01200BB0F0BD816E5A
:1097C000002917D00B8A112A28D19D420ED1019869
:1097D0001231093A01F09CFE012807D1BB59200043
:1097E0009D6EFFF70FFE29000200DEE73221200008
:1097F000FFF7D8FC2000FEF701FF061E1BD0416AD0
:10980000002918D00B8AAB4215D1082201981231D9
:1098100001F07EFE01280ED1716A0AE09D42E9D175
:1098200008220198123101F073FE0128E2D1BB59E0
:10983000996E8A7EB9E7200001F09AFDBCE7C04628
:109840000068FF1FF0B56B4D87007E5985B03378F7
:1098500002900393002B00D087E0B368346A019331
:109860007078062817D101221B7D134202D0217B7C
:10987000114218D10222134202D0217B114251D150
:109880000422134203D0237B134200D08BE0019BC0
:109890005A7DEB5991E007380428F8D801F0B8FD5B
:1098A000032E42678300B36E002B03D11C2001F00E
:1098B000FFFDB066EB599C6E002C1CD010220021DD
:1098C000200001F085FD0298FFF79CFD01002000BB
:1098D000FFF72DFA01F0DCFF208220000821123072
:1098E000FFF725FA0298FFF78DFDA076EB592100CE
:1098F000D888FFF70FFC0822EB591CE0B36E002B51
:1099000005D01A00198AF0881232FFF70DFC0222E6
:10991000019B197DEB5911423DD0207B10423AD07A
:10992000073208E0F488FCF7DBFD01002000FFF7B8
:1099300011FC0A22EB595A70029B9C002A59537859
:10994000073B042B11D8D088FEF758FE00284ED0D4
:10995000C3895A08D2182849029B0298CB542B5924
:1099600041180433254801F0A3FF05B0F0BDFCF712
:109970009FFD03000120834201D100200393EB5996
:10998000DE88FCF79BFD039902003000FFF7ECFB3B
:10999000019AEB59117D042211420CD0217B114216
:1099A00009D00B22C7E7F688FCF73CFD0100300028
:1099B000FFF7EEFB6BE7019A527D01210A4204D0CA
:1099C000607B084201D00C22B5E702210A4204D094
:1099D000607B084201D00E22ADE704210A4204D088
:1099E000627B0A4201D01022A5E71222A3E7FA22E5
:1099F0005200B0E70068FF1F0468FF1FBB9D001105
:109A000010B5064B1A780423100018401A4200D0F3
:109A10000348FFF727FA002010BDC0468D66FF1FE0
:109A20001845FF1F70B50400FFF7D4FA051E43D197
:109A30002000FFF77FFA234EA400A0598268937C90
:109A4000DB0708D50321036A1B790B40012B02D1E8
:109A5000017F0B430377431DD97F8B1E022B0DD84B
:109A6000022900D00121C088FCF790FF042133595E
:109A70001A7F59700A431A77280070BD01290CD14A
:109A800002231022437000210C3001F0A1FC305958
:109A900010213530FFF74BF9EEE70529ECD1022311
:109AA000D118437010220C3001F012FD04233259FA
:109AB000117F0B431377EAE708251828DCD1053D11
:109AC000DAE7C0460068FF1FF0B58BB00591438808
:109AD0007E4F9E00F45915000493002C15D10129E6
:109AE00002D000200BB0F0BD101D57781678FFF79C
:109AF00057F9EB68320002932B7A04990193009096
:109B00003B002000FCF70CFFEBE7E388049A93424C
:109B100001D00820E6E72378012B00D1D4E0059B93
:109B2000581E092800D9CFE001F072FC05CE0A29A1
:109B3000CC506C859AB229000498FFF773FFD1E7E7
:109B4000200029001022453001F0C2FCB9594B78A1
:109B5000042B02D1013B4B70C3E70B000A002533F5
:109B600035320C310498FFF795F90498FFF702FAA3
:109B70000522431E9841BB59C0005A70B2E720002D
:109B800029001022553001F0A3FC049B4F4C9D008E
:109B9000295904980A0006AB55320C31FFF77AF9BF
:109BA00029591022453106A801F0B2FC012808D13C
:109BB0000498FFF7F7F90590002804D106222B59E5
:109BC0005A7005988EE708230593FAE763780C2B03
:109BD0007AD1E36E002B03D11C2001F069FCE06612
:109BE000BB59D86E00286FD01022290001F070FCFC
:109BF000BB590498DC6EFFF705FC0D22A076BB591B
:109C00005A706EE7E06E00285ED063780D2B5BD152
:109C10002B8808220382A91C123001F059FCBB5981
:109C20009A68517D0222114226D0186A407B104268
:109C300022D00C32E4E763780E2B45D1236F002B42
:109C400003D1162001F034FC2067BB59186F00289F
:109C500003D01022290001F03BFC0F22BB59CFE7B3
:109C600063780F2B30D1206F0622691C103001F071
:109C70002FFCBB599A68517D0422114203D0196A06
:109C8000497B1142D5D100210498FFF78BFA28E7D0
:109C9000636F002B0DD0BB59586F0028F3D01022F2
:109CA000290001F015FC0122BB5952425B6F1A6179
:109CB000E9E7142001F0FCFBBB5960675B6F002BE8
:109CC000E9D126E72978DFE707200BE70068FF1FC7
:109CD00010B5064C207001F073FD06212078FDF7C9
:109CE00091FF0348FEF778FC10BDC0461368FF1FC4
:109CF000718E001100200BB270B50D00834216DA90
:109D0000264B187801F04CFD041E0DD00378922BE1
:109D10000ED0A02B37D0224B1878FF283AD0210044
:109D200001F09EFD002835D180200002684070BD02
:109D300043780E2B0BD03E2BEDD18378052B12D020
:109D4000082BE8D181798088FFF7D8FA08E0154B15
:109D500082889A42DFD183681878591CFEF7C0FECA
:109D6000002817D1D7E7104B1B785B0712D50F4B94
:109D70001B68002B0ED09B68002B0BD0C289811D65
:109D800080889847ECE7FFF741FAA068002801D0E7
:109D900001F0DEFD200001F033FBC5E71368FF1F73
:109DA0001145FF1F182000008D66FF1FFC67FF1F75
:109DB00010B50078FFF712FA10BD10B50078FFF764
:109DC000FDFA10BD0C234343084A10B59B185A688E
:109DD000002A03D0012901D1904710BD9B68002BB8
:109DE000FBD00029F9D19847F7E7C0463068FF1F3C
:109DF00001238340094A10B5946B1C439463506B54
:109E000098435063D46B20009843012901D120006E
:109E10001843D063116B0B43136310BD00800040E7
:109E2000F0B500240127154B85B0DA6B144E039270
:109E30001A6C0192DA64019BE3403B4217D0039D08
:109E4000E5403D400295E5B202992800FFF7BAFFD0
:109E5000316A736A002908D03900002B01D00299B9
:109E600079402800FFF7C4FF01E0002BF9D101344D
:109E70000C36172CDFD105B0F0BDC0460080004085
:109E80001468FF1F064B01215A68C2400A4204D0E1
:109E90001B68C3401800084070471B6DF9E7C046B7
:109EA000008000400122064B8240002903D0D9687F
:109EB0000A43DA607047D9689143D960FAE7C0462F
:109EC0000038004030B5032444430F4BE25C1B19BB
:109ED0009C785D7801232D1B0135AB40013BA340ED
:109EE000A140DB430C00122807D808499200521801
:109EF000116819402143116030BD054A11680B40BB
:109F000023431360F8E7C04637BC001108F0004057
:109F100014F00040C21F70B5D4B20623092C0BD830
:109F20000125084C9540002908D00021FFF7CAFF01
:109F300023682B4323600023180070BD2368AB43C4
:109F4000F8E7C04600380040214BF0B51B185B789D
:109F5000022B21D1032444431E4A1F4EA35C121935
:109F60009478012215008540B76B013CE4B23D4373
:109F7000A240B563194C122815D89B0000290CD1BA
:109F800017495B1899680A439A600123205C154AB7
:109F9000834011680B431360F0BD11495B18996849
:109FA00091439960F1E70E4B00290DD159690A439D
:109FB0005A61225C1328E8D00123203A93400A49D1
:109FC000086803430B60E7E7596991435961F0E77B
:109FD0001468FF1F37BC0011008000407CBC0011DA
:109FE00000F00040A0F00040A4F00040F8B50024CC
:109FF0001B4E1C4D1C4B1B5D012B1FD1194A926936
:10A00000E2401A420BD00122B25693402200143A89
:10A01000D2B2022A09D815494A6913434B61013467
:10A0200002360C35172CE5D1F8BD0022B2560F4987
:10A030009200521891680B439360F0E7022BEED127
:10A04000E7B23800FFF71EFF01235840C1B23800C5
:10A05000FFF77AFF3800FFF715FF6877DFE7C046A4
:10A0600009BC00111468FF1F1568FF1F00F00040B5
:10A07000012202388240054B002903D059690A4366
:10A080005A617047596991435961FAE700380040B5
:10A09000F8B50E0001210F008740114A0400D36873
:10A0A000FD43BB43D360831E8B4201D8FFF7E0FF23
:10A0B00000212000FFF72EFF0A4A0B4B5168012EAA
:10A0C00005D139431B1951605E700020F8BD29404D
:10A0D000516002221C1962709A6915409D61F4E773
:10A0E00000380040008000401468FF1F012210B5B6
:10A0F0008240074B002906D019680A431A600121E3
:10A10000FFF7C6FF10BD196891431960F7E7C04615
:10A11000008000400C2370B5002543430A4A290003
:10A120009B181D70094B04001B185D70FFF7B0FFF2
:10A130000123A340064928000A681A430A6005491A
:10A140000A689A430A6070BD3068FF1F1468FF1FD9
:10A15000348000403080004070B504000E00FF28BD
:10A1600013D003250540FFF7D5FF084AA3089B003D
:10A170009B183F22ED00AA40AE4019682000914391
:10A18000314319600121FFF78DFE70BD1838004082
:10A19000F8B50C244443134B0500E4186368002B06
:10A1A00003D1A3681220002B1AD0022201270E4BE4
:10A1B00000215B195A7028002770FFF769FF636858
:10A1C0001E1E08D0A3683E00002B04D02800FFF715
:10A1D00059FE4640F6B228003100FFF709FE002084
:10A1E000F8BDC0463068FF1F1468FF1FF7B5C420D4
:10A1F000FF222B4B80001958002491433F3A0A4319
:10A200001A508022274F5202274E1A60274B1D5D9D
:10A21000002D21D0A31E012B03D80121E0B2FFF7AE
:10A2200027FF012D18D11F4B9B69E3402B4213D010
:10A23000E3B218000193FFF725FE01000198FFF734
:10A2400055FFE3B2143B022B1DD801217156184A69
:10A250008D405369AB4353613B7F002B0DD0E5B27A
:10A260002800FFF795FF2800FFF70CFE7B7F010019
:10A27000834202D02800FFF7A5FD01340C370236D7
:10A28000172CC3D1F7BD012100237156F3568D4021
:10A29000074A9B009B189A68AA439A60DCE7C0466D
:10A2A00000E100E01468FF1F09BC00111568FF1FE2
:10A2B00000F0004010B501210400FFF7E9FE012382
:10A2C000044A002011194B70A34091690B4393611C
:10A2D00010BDC0461468FF1F70B50E0015000400C5
:10A2E000FFF718FF0C236343094A20009B189D6069
:10A2F0005E60FFF74DFFF021064B074A8900051EFF
:10A300005A5002D02000FFF705FF280070BDC0465C
:10A310003068FF1F0000FF1F219E001170B5134D14
:10A3200007202C78002C1FD19822210052002800F1
:10A3300001F006FA0123C420FF222B700C4B800091
:10A340001C635C630B4B1C605C600B4B19589143A6
:10A350003F3A0A431A50802252021A600D20074ADF
:10A36000074901F0FDF9200070BDC0461468FF1FC9
:10A3700000800040A0F0004000E100E0EDA10011ED
:10A38000ED9F0011030010B50620072B09D8054AE0
:10A39000137001F00DFAD7210020034B034A890006
:10A3A0005A5010BD4045FF1F0000FF1F151BFF1F27
:10A3B00070B51D0002240C2910D8094ACA40D207E2
:10A3C0000CD5FBF72FFF041E08D1059A049928002D
:10A3D000FBF744FFFCF7B2FDFFF712FB200070BD56
:10A3E0001210000030B50D7802232C009C43184257
:10A3F00001D02B431C0008252300AB43284201D089
:10A400002B00234320241D00A543204201D01C43E0
:10A4100025002A230D70184204D011781E3B0B43EF
:10A42000137030BD0028FCD10C2113788B43F7E763
:10A43000F8B51D0006AB1B88140007AA0E000B2000
:10A440001778002B27D10A78022A49D14A68507818
:10A4500011780002244A08438018042840D800F0EC
:10A46000D7FF03121D1B2300F06801F031FA021C14
:10A47000C0B2B84200D93A1CD2B22000F1682A809A
:10A4800001F026F806E00222F3681B882A80237078
:10A490001B0A63700020F8BD0622EEE701232B8023
:10A4A000F3681B782370F5E7F368002B16D00822B9
:10A4B0002A801A8822701A88120A62705A88A2703A
:10A4C0005A88120AE2709A8822719A88120A627176
:10A4D000DA88A271DB881B0AE371DBE72B80D9E7FE
:10A4E00001202B80D7E7C04600D6FFFFF7B5160046
:10A4F0000A781D0008AB1F880C000123022A18D11E
:10A500004A685078117800022B4A084380180328C3
:10A510000FD800F07DFF02254439E06801F0D8F93A
:10A52000C0B20723B84204D37B190193152B02DD77
:10A530000D231800FEBDE0682A003100C01900F0AC
:10A54000C7FF6B4600209B88E268D0541B4B1B68FA
:10A55000834203D01B68834200D098470023E8E77A
:10A560000B23002FE5D1022DE2D1737832781B0244
:10A570001343E2681380114B1B68002BEED01B685D
:10A58000002BEBD00120E8E70B23002FD1D1062DC3
:10A59000CED12A003100E06800F09AFFDEE70B23FD
:10A5A000002FC6D1012DC3D132787533012AC0D80E
:10A5B000E3681A70D2E7C04600D6FFFF206AFF1F8B
:10A5C00070B50C001500072837D800F021FF0414DF
:10A5D00036361B36242E182015290BD8184E162275
:10A5E0000021300000F0F4FE22002900300000F0CD
:10A5F0006FFF002070BD18200229FBD11288114B7B
:10A600001A80F6E718200829F4D10A000E4829001C
:10A6100000F0AEFFEDE718200129EBD10B4B1078CD
:10A620000B49DA69FFF7DEFEE3E718200129E1D1E3
:10A63000064B10780749DA6BF4E70220DAE7C046E8
:10A64000086AFF1FBE45FF1FB445FF1F4445FF1F9B
:10A650006C45FF1F8C45FF1F030010B50020DB0772
:10A6600004D50721024A034800F08CF810BDC0460B
:10A6700094BC00114445FF1F054A030010680028E0
:10A6800003D082889A4201D1806870470068F6E75B
:10A69000246CFF1F0A88030008009A4204D08A88AD
:10A6A00004309A4200D0002070470000F8B5F8222C
:10A6B00000230D4F0D4E79680500424333709942D7
:10A6C00000D07B600A4C0021200000F081FE0023B6
:10A6D0001A007C60AB4202D100203370F8BD013318
:10A6E0002280DBB2F834F5E7246DFF1F206DFF1FD9
:10A6F000286CFF1F73B56B46019006006846150075
:10A700001980FCF74DFF041E11D1002D0FD0768962
:10A71000002E11D00C2000F0CBFE00280ED0084AED
:10A720000460136886808560002B02D110602000D1
:10A7300076BD1A001B68F7E70224F8E71324F6E752
:10A74000246CFF1F012100220A4B10B549420A4C1C
:10A75000198099809A719A70084B20700120198095
:10A760005A60FFF7A3FF2078FCF778FF0448FDF755
:10A7700033FF10BD286AFF1F2C6DFF1F246DFF1FC4
:10A7800031A80011022310B5002802D0FFF7B2FF54
:10A790000300180010BD0000030010B50020DB0707
:10A7A00004D50421024A0348FFF7A4FF10BDC046A8
:10A7B000A8BC0011C445FF1FF0B50E2687B0039357
:10A7C0000CAB1F8802ABF61805000800310002929E
:10A7D000FDF768F804000120002C0FD03088FFF747
:10A7E0004BFF03000E20002B08D05E68002E05D022
:10A7F00021002800039B029A0097B04707B0F0BDE4
:10A800000A4B10B5984207D10122002352420A8018
:10A810008B708A808B7110BDFFF73CFF0028FAD047
:10A8200001235B42038000238370F4E7FFFF0000F5
:10A83000F8B5050001290AD1134E00243388F82702
:10A84000AB4219D028001149FFF7DAFF06E00229D0
:10A8500004D10139FDF73EFF0028EDD0F8BD3B00E3
:10A8600063437268D018D35A002B09D03A000021F4
:10A8700000F0AEFD0134E4B2054B1B78A342EED8E4
:10A8800001235B423380DDE7246DFF1F286AFF1F31
:10A89000206DFF1F10B5FFF7FDFE0300002083426F
:10A8A00000D0987810BD0000F0B589B01C000EAB48
:10A8B00080CB03901E8810AB1B78049202930B7A16
:10A8C0000D00DB0616D42B780593022B24D00498B8
:10A8D000FFF7D2FE002812D003689C46002B0ED052
:10A8E000029B2200019329003B00644603980096D6
:10A8F000A04705E00498FFF7BFFE002802D10E2014
:10A9000009B0F0BD8368002BF9D00A222900039812
:10A9100098470028D7D0F3E76B6858781A786B4BC4
:10A92000000210439842D2D8043B984210D2684BA0
:10A93000984242D015D8674BC0180128C7D80B20C1
:10A94000002EDDD1EB681A7859683A80200028E0A3
:10A95000614BC018032800D979E000F059FD846AE2
:10A96000789E5E4B9842B2D10B20002EC8D10123B5
:10A970003B80EB6831001B7823706889013080B21E
:10A98000FCF790FF3A88031E0ED0017802328A1835
:10A990003A80428962704289120AA270596802782C
:10A9A000E01C00F095FD06E004323A8031000422FC
:10A9B000601C00F00DFD0020A2E70B20002E9FD1AF
:10A9C000EB6807A91E8804233B80330A30002670F9
:10A9D0006370FCF767FF051E28D004AB9A890E232D
:10A9E00004A95B183E49C668FCF7D0FF00280BD1CC
:10A9F0002B783C486A680599FBF786FB002803D151
:10AA0000012304AA5B42D3813278022A06D17168FD
:10AA1000201D00F05DFD3B8802333B800E2304AA1D
:10AA20009B181B88A3701B0AE370C4E704ABDE818C
:10AA3000F4E70B20002E00D062E7E9680398FFF7E7
:10AA400029FF02233B802070000A6070B3E70B20CF
:10AA5000002E00D054E70222EB681B883A80237056
:10AA60001B0A6370A7E7E86800F032FFC2B2030078
:10AA70000720B24200D243E70DD00299DBB2711831
:10AA8000994202DB921BD3B20293029BE9681A003F
:10AA90003B8089195AE70023F6E70B20002E00D0EF
:10AAA0002EE70722EB683A801A7822705A78627093
:10AAB0005A88A2705A88120AE2701A792271DA88CA
:10AAC0006271DB881B0AA37175E7C0460429000088
:10AAD0000228000000D8FFFFFFD6FFFF0328000078
:10AAE000FFFF0000D8BB0011F0B58DB06B46002011
:10AAF000089120229B5E83423DDAA64B187800F035
:10AB00004FFE071E32D00378B02B2CD100790238CB
:10AB100016281FD800F01CFD17001E001E001E0086
:10AB200031001E0096001E001D011E0052011E0075
:10AB300073011E00CD011E0050021E001E001E00EB
:10AB40008E021E00E302944B94491B8878880B8088
:10AB5000FBF71AF83800FCF79BFF914B1B68002BA2
:10AB600001D038009847380000F04AFC8020089B4C
:10AB70000002434018000DB0F0BDF62200218748C6
:10AB800000F026FC0BAA3B7B7989388900923A00B9
:10AB90000D32FCF79FFD0400804B1B78002C3FD149
:10ABA00046E0804B788805937F4B4100CB5A0BAE33
:10ABB000073BDBB232880293002301937B4B2100D9
:10ABC00006930093059BFFF76FFE744D002810D18C
:10ABD000069B3A8A1B889A420BD13800059912309D
:10ABE00000F096FC002804D02B7862899B00EB18BB
:10ABF0005A80162306A81B18328820007989FCF792
:10AC0000C5FE2B7804009A00AA1851880029C3D0E9
:10AC10000133DBB22B70002807D006A9C98A9180C6
:10AC2000634A12889A42BCD802E0012149429180CD
:10AC3000002B04D059497888FAF7DAFF8AE73E8971
:10AC40000A2479E000253E89574B06937B88069AB3
:10AC50005B009B5A033B9D4202DB002DF0D05BE082
:10AC6000162206A812183B7B798900923A00300020
:10AC70000D32FCF72FFD0590002858D04689017A47
:10AC80007888FCF7F1FC041E44D1464B7888079382
:10AC9000069B4100C95A454B0439C9B206AAD28A5B
:10ACA00006930291019400930599079BFFF7FCFD21
:10ACB000041E2FD1069B39491A88931C002D26D1DA
:10ACC0004B807988384B4900CB5A5119033B8B4252
:10ACD00020DD059B31485B8941190B71A91C0135A9
:10ACE000C9B2EDB2059145191B0A2B71059B2D497F
:10ACF0000433181800F0ECFB2C4B059A1B88D31872
:10AD0000DDB22C4B9E4205D00136B6B29CE7498895
:10AD10009942D6D0002D0CD0204C2800618800F03C
:10AD20004FFC207021007888FAF772FF12E7059C2B
:10AD3000F0E7002C00D183E77B78142B00D109E7E2
:10AD400016493B794E800B700C717888FAF712FF28
:10AD500000E7162406ABE41821003889FCF7A2FDB1
:10AD6000011E00D1B7E1788822880F4C45002C5B8A
:10AD70000A4D013CE4B2029400240F4B019400956B
:10AD8000FFF792FD041E00D014E129007888FAF73D
:10AD90004FFFDFE62C6DFF1FB044FF1F306AFF1F1F
:10ADA000246AFF1F2A6BFF1F6066FF1F206CFF1FB6
:10ADB000AE44FF1FFFFF0000326AFF1F162406ABE0
:10ADC000E41821003889FCF76DFD011E00D182E1F5
:10ADD00078882288AE4C45002C5BAE4D013CE4B235
:10ADE00002947C89AC4B01940095FFF75DFD041E35
:10ADF00000D0DFE029007888FAF724FFAAE60025D2
:10AE0000A44B1D803B00FE331B78A24A7888079232
:10AE1000AB4208D99E4B12880693069943005B5AB1
:10AE2000013B9A4203DB0799FAF716FF92E61624D4
:10AE30006B00FB18059306ABE418059B21001889ED
:10AE4000FCF730FD011E03D1059B01241E8973E729
:10AE50007888924B2288069C099343001B5B904E96
:10AE6000013BDBB20293002300960193099BFFF79D
:10AE70001BFD041E02D0059B1E895DE77B88069A98
:10AE80005B009B5A079A108832881218934202DCA2
:10AE90001B1A013B33807F4C02303288099900191C
:10AEA00000F016FB2388328801359B182380EDB211
:10AEB000A8E70BAA3B7B7989388900923A000D32CA
:10AEC000FCF708FC00250590059B002B04D10A2403
:10AED000002D00D16EE060E0059B7888197AFCF7C0
:10AEE000C3FB0100041E63D1694C6C4B7888069447
:10AEF0000993069B4400E45A694B063CE4B20BAE4E
:10AF0000328807930294019100930599099BFFF7FA
:10AF1000CBFC041E4CD1079B5E491B881A1D002DDB
:10AF200030D14A80059B5B4C5A8963191A716B1C9E
:10AF30009BB2E318120A1A71162306A832881B184E
:10AF400079890598FCF722FDFF21AA1C2E1D0335E7
:10AF50000B00059092B2B6B2ADB2002803D006AB9A
:10AF6000DB8AD9B21B0AA218651911712B714C4DDD
:10AF7000301D2A884949201800F0AAFA2B88F618B3
:10AF8000B5B2A1E74988914207D17A880699520063
:10AF9000525AEB18053A9A42C4DC3E4C28006188AC
:10AFA00000F066FC207021007888FAF75FFED1E59A
:10AFB000002DF2D13E89BFE6162606ABF618310009
:10AFC0003889FCF76FFC3D000400FF3500282DD0C8
:10AFD000037A9B060CD400227B89398978880092F9
:10AFE0003A000C32FFF7E8FB041E10D03E8915E052
:10AFF0003088FFF741FB00281AD08368002B17D058
:10B000002100122278889847041EE4D0EEE7AB783E
:10B01000002B02D17888FAF739FE0026AB78002B96
:10B0200000D097E5002C00D194E585E60124DDE70A
:10B030000E24DBE7162506ABED1829003889FCF74E
:10B0400031FC041E47D0037A9B0611D4154A7B8835
:10B050001188994203D01448814207D11380134BC1
:10B06000F8261D780023D9B2A94221D30924A1E7EB
:10B070002888FFF701FB00282FD08368002B2CD0F5
:10B080002100122278889847041EDFD092E7C0463C
:10B090006066FF1F306AFF1F326AFF1F2A6BFF1FA7
:10B0A000206CFF1F246DFF1FFFFF0000206DFF1F9E
:10B0B00031005943546801336018615A0029D2D1D4
:10B0C0003C0008342100F82200F002FA21007888C0
:10B0D000FAF7E4FD3EE501246CE70E246AE71D4B18
:10B0E0001A887B889A4231D07888FAF7E1FD31E5F9
:10B0F000F823059851684343CD18C95A00291FD039
:10B100003B7A012B0BD16C88AB887888AA1D009400
:10B11000FFF752FB041E02D000233B722E88F82258
:10B120000021280000F054F900232B80059B0133F7
:10B13000DBB20593084B05991B78064A8B42D7D89A
:10B1400001235B421380002CCED0F5E500263400AD
:10B150000596EFE7246DFF1F206DFF1F70B50400FB
:10B160000E001500FFF796FA031E08D131000548BE
:10B17000FFF790FA03001120002B02D01C80002062
:10B180009D7070BDFFFF0000F8B50B4F06003B78C7
:10B190000D001400FF2B0ED00A2000F039FA011E1A
:10B1A00009D0B1230380002346800371C580048148
:10B1B000387800F055FBF8BD0546FF1FF7B50F00C6
:10B1C00008A90600088809A90B240988002821D1AC
:10B1D0000234022B1ED1557813782D021D432B000B
:10B1E0008B4301937334002B14D1FB68300019009A
:10B1F0000093FFF74FFB019C85420BD02A003000E3
:10B200000099FFF7ABFF041E04D12A0030007989B2
:10B21000FFF7BAFF2000FEBDF0B50E7885B00390B1
:10B220000AA805880120022E0DD14C682778647881
:10B2300024023C43054FBC4205D10398DBB2019682
:10B240000095FFF7BBFF05B0F0BDC0460229000026
:10B2500010B504000C4800F0C3F90C48A16B00F0D5
:10B26000BFF90B48E16B00F0BBF90A48216C00F014
:10B27000B7F9094B0948196800F0B2F9084B1B6887
:10B28000002B00D09847FEE7AABA0011C0BA0011FF
:10B29000CFBA0011DEBA001104ED00E0EDBA0011E2
:10B2A000306DFF1F002307B501A80193FFF7D0FF02
:10B2B000044A0548002110B5121A00F089F8F8F781
:10B2C0007FFBFEE7346DFF1F0846FF1F00000000F4
:10B2D00001B40248844601BC604700BFF94C01003C
:10B2E00001B40248844601BC604700BFEDA50000E0
:10B2F00001B40248844601BC604700BF55490100C3
:10B3000001B40248844601BC604700BF2526000006
:10B3100001B40248844601BC604700BF090E00002A
:10B3200001B40248844601BC604700BF055E0000CE
:10B3300001B40248844601BC604700BF7D37FF1F4F
:10B3400001B40248844601BC604700BFC51D00002F
:10B3500001B40248844601BC604700BF21240000BC
:10B3600001B40248844601BC604700BF017F000071
:10B3700001B40248844601BC604700BF091B0000BD
:10B3800001B40248844601BC604700BF7D18FF1F1E
:10B3900001B40248844601BC604700BF953BFF1FD3
:10B3A00001B40248844601BC604700BFA532FF1FBC
:10B3B00001B40248844601BC604700BFAD3AFF1F9C
:10B3C00001B40248844601BC604700BF291C00004C
:10B3D00001B40248844601BC604700BF154D01001E
:10B3E00001B40248844601BC604700BF45500000DC
:10B3F00001B40248844601BC604700BF35550000D7
:10B4000001B40248844601BC604700BF434D0100BF
:10B4100001B40248844601BC604700BFD13CFF1F15
:10B4200001B40248844601BC604700BF6532FF1F7B
:10B4300001B40248844601BC604700BFC9A90000AE
:10B4400001B40248844601BC604700BFED4A0100D8
:10B4500001B40248844601BC604700BFB14E000001
:10B4600001B40248844601BC604700BFCD34FF1FD1
:10B4700001B40248844601BC604700BFBD3CFF1FC9
:10B4800001B40248844601BC604700BF8D34FF1FF1
:10B4900001B40248844601BC604700BF8D12000021
:10B4A00001B40248844601BC604700BF014C010062
:10B4B00001B40248844601BC604700BF3D4B010017
:10B4C00001B40248844601BC604700BFD91B00009C
:10B4D00001B40248844601BC604700BFE94C01004A
:10B4E00001B40248844601BC604700BF7530FF1FAD
:10B4F00001B40248844601BC604700BFF539FF1F14
:10B5000001B40248844601BC604700BF5D170000DB
:10B5100001B40248844601BC604700BFCD4C010025
:10B5200001B40248844601BC604700BF1D36FF1FBE
:10B5300001B40248844601BC604700BF8B52010041
:10B5400001B40248844601BC604700BF4D1F0000A3
:10B5500001B40248844601BC604700BFE53CFF1FC0
:10B5600001B40248844601BC604700BF691F000067
:10B5700001B40248844601BC604700BF810E000050
:10B5800001B40248844601BC604700BF5522000058
:10B5900001B40248844601BC604700BFE9280000AE
:10B5A00001B40248844601BC604700BF5952010003
:10B5B00001B40248844601BC604700BF851F0000FB
:10B5C00001B40248844601BC604700BF350E00004C
:10B5D00001B40248844601BC604700BF51470100E6
:10B5E00001B40248844601BC604700BFE53A01004F
:10B5F00001B40248844601BC604700BF311B000013
:10B6000001B40248844601BC604700BFA54F010059
:10B6100001B40248844601BC604700BF1D4D0100D3
:10B6200001B40248844601BC604700BF2D35FF1FAE
:10B6300001B40248844601BC604700BF11470100C5
:10B6400001B40248844601BC604700BF7138FF1F47
:10B6500001B40248844601BC604700BF5118FF1F77
:10B6600001B40248844601BC604700BF193BFF1F7C
:10B6700001B40248844601BC604700BF4551010047
:10B6800001B40248844601BC604700BF85520100F6
:10B6900001B40248844601BC604700BF2539FF1F42
:10B6A00001B40248844601BC604700BFADAE000053
:10B6B00001B40248844601BC604700BF9DA9000058
:10B6C00001B40248844601BC604700BF1D4B010025
:10B6D00001B40248844601BC604700BFE117000086
:10B6E00001B40248844601BC604700BFC521000088
:10B6F00001B40248844601BC604700BFF30E00005D
:10B7000001B40248844601BC604700BF056A0000DE
:10B7100001B40248844601BC604700BF21460100D5
:10B7200001B40248844601BC604700BF0D520100CD
:10B7300001B40248844601BC604700BF75A90000FF
:10B7400001B40248844601BC604700BFB70E000048
:10B7500001B40248844601BC604700BF2D3AFF1F78
:10B7600001B40248844601BC604700BFED32FF1FB0
:10B7700001B40248844601BC604700BFA137FF1FE7
:10B7800001B40248844601BC604700BF5125000057
:10B7900001B40248844601BC604700BF0124000098
:10B7A00001B40248844601BC604700BFF54E010069
:10B7B00001B40248844601BC604700BF151BFF1F4F
:10B7C00001B40248844601BC604700BFC92600009E
:10B7D00001B40248844601BC604700BF4D32FF1FE0
:10B7E00001B40248844601BC604700BF156B0100EC
:10B7F00001B40248844601BC604700BFE548000030
:10B8000001B40248844601BC604700BF01890000C2
:10B8100001B40248844601BC604700BF79180000AB
:10B8200001B40248844601BC604700BFC13BFF1F12
:10B8300001B40248844601BC604700BFC94A010008
:10B8400001B40248844601BC604700BF6DBC0000E3
:10B8500001B40248844601BC604700BFE139FF1FC4
:10B8600001B40248844601BC604700BF594F010043
:10B8700001B40248844601BC604700BF090E0000C5
:10B8800001B40248844601BC604700BFC95C0100A6
:10B8900001B40248844601BC604700BF2951010041
:10B8A00001B40248844601BC604700BFB54C0100AA
:10B8B00001B40248844601BC604700BFA9460100AC
:10B8C00001B40248844601BC604700BFDD66010048
:10B8D00001B40248844601BC604700BFDD5201004C
:10B8E00001B40248844601BC604700BF3D18000017
:10B8F00001B40248844601BC604700BFC53F000058
:10B9000001B40248844601BC604700BF456B01009A
:10B9100001B40248844601BC604700BF6D3AFF1F76
:10B9200001B40248844601BC604700BF6571010054
:10B9300001B40248844601BC604700BFC56D0100E8
:10B9400001B40248844601BC604700BFB352010005
:10B9500001B40248844601BC604700BFD9490100D8
:10B9600001B40248844601BC604700BFC130FF1FDC
:10B970000002010302030303040305020602070297
:10B98000080209000A030B030C020D000E030F034B
:10B99000100311031303140315001600A53D001135
:10B9A000D93D00110000000002000000B2B90011F2
:10B9B000192A0F180A000000F1590000FD240000A8
:10B9C00041460100E17C0011F59C00114971001114
:10B9D000E57A0011F1520011E9AA0011654F00113A
:10B9E0009D3F0011CD400011000000001616000020
:10B9F00002000000FCB90011F4FFF3FFD2FC0000CC
:10BA00000D42001100000000000000005475796133
:10BA10000042312E33003030303100676974687570
:10BA2000622E636F6D2F7076767800425448303105
:10BA3000000000000200000048BA0011292A282A4C
:10BA4000272A262A252A242A0A180000E2040000B0
:10BA50007102000078EC0000744000001027000024
:10BA600060F0000006640000204E000000000000AE
:10BA7000050000001F501D00023CB400000114002E
:10BA80001300000081020000303132333435363784
:10BA90003839414243444546005048592B363258C4
:10BAA00058504C555330353034005B486172642037
:10BAB0006661756C742068616E646C65725D0A0005
:10BAC0004C522020203D203078253038780A005014
:10BAD000432020203D203078253038780A0050530C
:10BAE0005220203D203078253038780A00494353D1
:10BAF00052203D203078253038780A00F556001164
:10BB000049570011000000000200000014BB0011A2
:10BB10006F2A6E2A1A18000001A000000000000021
:10BB20006410B71DC8206E3BAC30D9269041DC763E
:10BB3000F4516B6B5861B24D3C7105502083B8EDE8
:10BB400044930FF0E8A3D6D68CB361CBB0C2649B0C
:10BB5000D4D2D38678E20AA01CF2BDBDFB349B5F31
:10BB60008000008000100000000000004B5D00110C
:10BB7000D57300116F5D0011DD770011F35D0011C9
:10BB8000B3770011695E001189770011BB5E001167
:10BB900051790011235F001151790011555F001197
:10BBA0000B790011695E001141770011E15E00110F
:10BBB000E97800110000000000000000C75F0011DC
:10BBC000E978001129600011ED730011052A042A9B
:10BBD000012A002A02290328012800280118001838
:10BBE00000000000000000000000000000000087CE
:10BBF0000101020102010102010203030401030128
:10BC0000010101010303020103000D000E001000F9
:10BC1000110013001401070108010A010B011C01A6
:10BC20001D02040205020702080219021A021C0280
:10BC30001D030103020317000201000504000807A9
:10BC4000000B0A001716001D1C010201010504016A
:10BC50000E0D011110011413011716011A19020219
:10BC600001020B0A020E0D02111002141302171624
:10BC7000030504030807030B0A030E0D000102036A
:10BC800007090A0B0E0F101112141718191A1B1F8F
:10BC90002021220031A40011EDA4001100000000B9
:10BCA00002000000DEBB00110000000019B200110C
:0CBCB0000000000002000000DCBB0011DE
:020000041FFFDC
:1000000000000000013F0011B8B90011B4B900119F
:100010001463FF1F0000000000000000000000004B
:1000200000000000000000000000000000000000D0
:1000300000000000000000000000000000000000C0
:1000400000000000000000000000000000000000B0
:1000500000000000000000000000000000000000A0
:100060000000000000000000000000000000000090
:100070000000000000000000000000000000000080
:100080000000000000000000000000000000000070
:100090000000000000000000000000000000000060
:1000A0000000000000000000000000000000000050
:1000B0000000000000000000000000000000000040
:1000C0000000000000000000000000000000000030
:1000D0000000000000000000000000000000000020
:1000E0000000000000000000000000000000000010
:1000F0000000000000000000000000000000000000
:1001000000000000000000000000000000000000EF
:1001100000000000000000000000000000000000DF
:1001200000000000000000000000000000000000CF
:1001300000000000000000000000000000000000BF
:1001400000000000000000000000000000000000AF
:10015000000000000000000000000000000000009F
:10016000000000000000000000000000000000008F
:10017000000000000000000000000000000000007F
:10018000000000000000000000000000000000006F
:10019000F134FF1F3933FF1FC1660100000000006A
:1001A000000000000000000000000000000000004F
:1001B000000000000000000000000000000000003F
:1001C000000000000000000000000000000000002F
:1001D000000000000000000000000000000000001F
:1001E000000000000000000000000000000000000F
:1001F00000000000000000000000000000000000FF
:1002000000000000000000000000000000000000EE
:1002100000000000000000000000000000000000DE
:1002200000000000000000000000000000000000CE
:1002300000000000000000000000000000000000BE
:1002400000000000000000000000000000000000AE
:10025000000000000000000000000000000000009E
:10026000000000000000000000000000000000008E
:10027000000000000000000000000000000000007E
:10028000000000000000000000000000000000006E
:10029000000000000000000000000000000000005E
:1002A000000000000000000000000000000000004E
:1002B000000000000000000000000000000000003E
:1002C000000000000000000000000000000000002E
:1002D000000000000000000000000000000000001E
:1002E000000000000000000000000000000000000E
:1002F00000000000000000000000000000000000FE
:1003000000000000000000000000000000000000ED
:1003100000000000000000000000000000000000DD
:1003200000000000000000000000000000000000CD
:1003300000000000000000000000000000000000BD
:1003400000000000000000000000000000000000AD
:10035000000000000000000000000000000000009D
:10036000000000000000000000000000000000008D
:10037000A5B2001100000000000000000000000015
:10038000000000000000000000000000000000006D
:10039000000000000000000000000000000000005D
:1003A000000000000000000000000000951AFF1F80
:1003B000000000000000000000000000000000003D
:1003C000000000000000000000000000000000002D
:1003D000000000000000000000000000000000001D
:1003E000000000000000000000000000000000000D
:1003F00000000000000000000000000000000000FD
:081838004071FF1F4118FF1F62
:10184000024981F3088802F0CFFC00004071FF1FBD
:1018500010B502F0B1FB072804D0122808D00228E6
:1018600008D010BD044A0420136B01331363F8E75A
:101870000220F6E71420F4E70867FF1FF8B5070019
:101880000C0026002500503630785135002804D150
:101890000300287058342370F8BD2978CA00481E08
:1018A0008141A3183800A25C5B68C9B2FFF7D0FF82
:1018B00000280DD12B78DA00A218013350602B706C
:1018C0003378044A013B3370136A01331362D8E75B
:1018D0000123DFE70867FF1F5C234343074910B577
:1018E000C9180B0058331B78012B05D1FFF7C6FF31
:1018F000034A936A0133936210BDC0463C67FF1FE1
:101900000867FF1F10B502F0BFFB064A0121130054
:1019100010CB4942D967044B136002F035FC20001C
:1019200010BDC04600E100E01000100010B504003A
:1019300002F0AAFB024B1C6002F026FC10BDC04660
:1019400000E100E010B5040002F09EFB4021094ACE
:10195000200013688B43136002F03EFB01F0AAFDE8
:101960000022054B01201A60044B04321A6002F079
:10197000C3FBFEE71CF00040C4F00040C0F0004094
:10198000431E5A425341A022F0B5D2015B4213409C
:10199000154D164A40019B182A18127E8BB00191F2
:1019A000002A1BD01A000832D46F0022E6B206AF1C
:1019B000E4B294420EDC2818C369002B08D00199C8
:1019C00002AA117106AA049202AA167303A89847E4
:1019D0000BB0F0BD1978B9540132EAE71A7D1A78D4
:1019E00006AB01261A70E6E7C869FF1F00400040F9
:1019F000F0B5254B04004001C25C85B0002A2BD015
:101A00001A18117E002927D0917E002924D011793F
:101A1000022921D11689D788D168F51BADB22A1CBD
:101A2000102D00D9102292B2BE4217D118180123EE
:101A300003710023C269C38003819A4206D06846BD
:101A4000032103730171029301A890470820002C21
:101A500000D0192001F026FC05B0F0BD013C654224
:101A60006C41A0256442ED012C40084D1B186419FF
:101A7000074D0633013A92B2AA42EDD01888461CAF
:101A80001E80085C2070F5E7C869FF1F0040004019
:101A9000FFFF00000F220E4B10B59868104002386F
:101AA0000A280BD802F014F90D0A0B0A0A110A0AC7
:101AB0000A0A060002210020FFF762FF10BD012183
:101AC000F9E70020FFF794FFF8E7DB6FF6E7C04681
:101AD000004000400F220E4B10B5986810400238AD
:101AE0000A280BD802F0F4F80E0A0B0A0A120A0AA6
:101AF0000A0A060002210120FFF742FF10BD012162
:101B00000800F9E70120FFF773FFF7E7DB6FF5E760
:101B10000090004013B5334C2378072B3DD8324B4F
:101B20001A78324B002A39D18022196852020A43AE
:101B30001A60252001F07AFF20232D4A11680B43FB
:101B4000802113606B460422C905086807331042E0
:101B500028D080210422C905C86810422ED08021D7
:101B60002020C905CA688243CA6014221A701A78F4
:101B7000002A2FD18021C905C86820320243CA60DB
:101B800014221A701A78002A28D11A4B1A7D22784A
:101B90005A601D221A705932DA6013BD1A6816494C
:101BA0000A40C5E7086802430A6014221A701A78CE
:101BB000002ACED01A78013AD2B2F7E7C8680243B9
:101BC000CA6014221A7019784A1ED2B21A700029FB
:101BD000F9D1C4E71A78013AD2B2C7E71A78013AC4
:101BE000D2B2CEE74045FF1F0846FF1F3CF0004041
:101BF0003845FF1F00200040FFFFFEFF564B70B529
:101C00001B68012B03D1554A936D0133936502F094
:101C100093F8534B534A1860534B544C1A600123AA
:101C2000534A1360534A13602378002B06D00622D0
:101C30005149524802F058F900232370504A514B41
:101C400010681B78C1B2002B0ED14F4CC0B2237864
:101C50005BB2002B4FDB237824785BB264B21B04A9
:101C600024021B191B1813600B1C50294ED950233A
:101C7000464A47491078DBB2FF2202284BD1086858
:101C8000444C454D267890432A78964254D9227880
:101C900024782E78023B5D10A31B6B435201D31AAC
:101CA00010335B111843086002F0B6F9031F012BD3
:101CB00045D83A4B1B78002B06D0394B1B78002BAC
:101CC00002D0002002F088FAA122364B92009978C7
:101CD000354B4A431B689B18832292009B181B7844
:101CE000033B012B03D8AF20400002F035F801225E
:101CF0002E4BDA8270BD237824785BB264B2FF3356
:101D0000FF341B0424021B190138ABE7CAB2022AB4
:101D1000AED20223ACE70868254C264D26789043C6
:101D20002A78964208D9227824782D78023B5B10D5
:101D3000641B63435201B2E72378DBB2B2E70228A7
:101D4000D5D11D4B1B78013B022B03D91B4B1B78B4
:101D5000022BCCD16C20C8E79809FF1FFC0FFF1F96
:101D60004066FF1FFF3F0000141003404466FF1F42
:101D70000C10034000100340D50BFF1F7211FF1F12
:101D8000B40003408C09FF1F680AFF1F490AFF1FA8
:101D900094000340460AFF1F470AFF1FF908FF1F70
:101DA0002209FF1F300DFF1F3409FF1FBC0BFF1F4F
:101DB000440AFF1F450AFF1F1C09FF1F2309FF1FBD
:101DC00010B502F001FA0022014B1A8010BDC04686
:101DD0003C66FF1F10B502F067F9A121054A890092
:101DE0009478054A61431268044B5218528C1A8049
:101DF00010BDC046300DFF1F3409FF1F3C66FF1F9A
:101E000010B50D4B0D4A9978A1239B004B431268E6
:101E1000D218531DD97F0A4B1B88994209D2441C02
:101E200007D0C82805D0D2695B1A5A43054B5343E3
:101E3000C01802F0D9F810BD300DFF1F3409FF1F84
:101E40003C66FF1F7102000070B5244D2B68002B0B
:101E500028D002F059F82B68D8402B680400002BDA
:101E600027D002F079F82B68D8401D4B1D4A99788D
:101E7000A1239B004B431268D118D25C91239B0095
:101E8000002A20D0CA580132CA50174B17491B6884
:101E90000868834214D3D23B181A012A1AD0144B73
:101EA000186070BD02F030F8124B196802F0C4F8E7
:101EB000D3E702F051F80F4B196802F0BDF8D4E7F0
:101EC0000D495B18E8E7CA500C4B1B68DB68E41847
:101ED000201AE4E7F530FF30E1E7C0461C08FF1F99
:101EE000300DFF1F3409FF1F9C09FF1F4066FF1FB5
:101EF000A009FF1F1808FF1F2DFF3F004866FF1FA6
:101F000070B504000D00282916D10300A433C2883F
:101F10001B889B1A0B4A9BB293420DD906006A3666
:101F200005223100653001F0FFFF002804D13100A7
:101F3000200001F039FF70BD2900200002F014F9E3
:101F4000F9E7C046FE7F0000F8B50400012001F06B
:101F500033FF02F0C1F80300184A19491060886A7B
:101F60008D6AA842FBD1174D174E28607568AC46A4
:101F7000164D2F680025BC4501D275687D1B144E97
:101F800000193560C862A4204C6A400320434862AF
:101F900010490978002905D00F490978022902D192
:101FA0000F3B1360F8BD012901D1083BF9E7032974
:101FB00001D1053BF5E7033BF3E7C046E408FF1F0B
:101FC00000F00040340AFF1F28100040180AFF1FCD
:101FD0001C0AFF1F1C09FF1F4A0AFF1F70B580243F
:101FE0001025E405A3682B43A36001F0ADFEA368B0
:101FF000AB43A36070BD0000F7B5160080221C0043
:102000001023D2050191916805000B4393600022D3
:102010005A4BD7301A6002F017F89D232A002F0080
:102020009B00EB58CA3201210092FC37002B01D0F3
:102030000021009A386802F0E7F82900009BCB31B4
:102040001A784F4BD3351A604B780A781B0213432A
:102050008A7812041A43CB781B061343494A1BBAE9
:1020600013604B790A791B0213438A7912041A43CD
:10207000CB7931001B061343434A1BBA13606B78BC
:102080002A781B021343AA7812041A43EB781B0622
:1020900013433E4A1BBA1360019A330213433C4A6E
:1020A00013603C4B22001B1B9C4603293DDCB308FC
:1020B0009A0013005142B21A032A46D1354AE01859
:1020C000511A82784078120400020243E05C043323
:1020D00002430A600022FF2B4BDDF0222E4B12013F
:1020E0001A600F222D4B1A602D4A1368002BFCD06A
:1020F0000023224A27491360091B321D0B191B6854
:10210000043A180A23706070180C1B0EA070E3705C
:102110000434002AF2DC802210213B68D20501330E
:102120003B6093688B439360F7BD6346D5789818FE
:1021300093782D061B042B43157804392B435578CF
:1021400004322D022B430360AFE7022A0AD1114A61
:10215000E05C511AE2185278120202430A6004331A
:102160009BB2B7E7012AB5D10A4A521AE15C116065
:10217000F5E7084959180A600433ACE70000044049
:102180003C00044038000440340004403000044067
:102190000C0004400001044004000440100004400E
:1021A00014000440F7B5150080221C001023D2054E
:1021B0000091916807000B4393600023654AD73074
:1021C000136001F041FF9D233E009B00F9583B0046
:1021D000CA363200FC33002900D07FE0586802F094
:1021E00013F8390032785C4BCB311A604B780A789F
:1021F0001B0213438A78AC4612041A43CB78281D7D
:102200001B061343554A1BBA13604B790A791B020C
:1022100013438A7912041A43CB791B061343504A9D
:102220001BBA13604B7A0A7A1B0213438A7A120490
:102230001A43CB7A21001B0613434A4A1BBA136088
:10224000009A2B021343484A13602200474B1B1B82
:102250000093009BCE785B1801938B7836061B04A5
:1022600033430E78043833434E7804313602334317
:10227000019E33600328ECDC0321A808431C9B006B
:102280002940800003292BD13849E5185E18A97828
:102290006D78E35C09042D02294319433160030082
:1022A00008330021FF2B2DDD314B324919600F21FE
:1022B000314B1960012327490B60304B1968002905
:1022C000FCD006211B680B40042B20D0802200206C
:1022D000D20593680A318B439360FEBD01217DE7EF
:1022E000022908D121495D18E1184978E35C090207
:1022F00019432960D3E70129D3D11C495918E35C5C
:102300000B60CCE71948181801600433CAE70023B2
:1023100010490B606346002B0CDC3B00FC335A6811
:10232000102101325A608022D205936801208B432C
:102330009360D2E7009B9B181B68190A13705170B9
:10234000190C1B0ED37004235B4291709C44043221
:10235000E0E7C046000004403C0004403800044070
:1023600034000440300004400C00044000010440EC
:1023700004000440080F0000100004401400044052
:1023800070B5061E19D00222614B9B799343012B35
:1023900013D1604B1A78FF2A0FD15A78FF2A0CD13B
:1023A0009A78FF2A09D1DA78FF2A06D11A79FF2A0A
:1023B00003D15B79FF2B00D1A7E0574B0C201A7893
:1023C000012A08D00022554D1A702B781A00093ABC
:1023D000042A01D8212070BD5A1F012AFAD94C4C79
:1023E000A07B042800D990E0A279032A00D98CE0D0
:1023F000821E012A03D862881F2A00D885E0002E99
:1024000061D0012E00D080E0A288012AE2D0002B0A
:102410000AD10138032803D801F05AFC151D1915FB
:102420001F202E7001F0D8FC2B785A1E032A16D8D4
:1024300000253B4B1D602823237501F0C5FCA842F5
:102440002ED0A580C6E7022320202B70EAE70423C4
:1024500022202B70E6E7032321202B70E2E7073BC5
:10246000012BB7D82F4B1B68DB6A9B06B2D52E4BCE
:102470001A78002AAED1A27B911E012901D9002A27
:10248000A8D1022280211A702823284D890128789A
:10249000237501F0E9FC80212878890101F0B4FD61
:1024A0000123A380224B1B78002B0AD0FA22802123
:1024B000204B92001B8809025A431C4B187801F0EC
:1024C000ABFC002087E701F0DFFD2B78A680073BFF
:1024D000012B06D918482E7001F0E6FC1E2001F0F1
:1024E0007BFC114B114C1A78002A06D08021002267
:1024F000207889011A7001F0B7FC01F045FE8021B7
:102500002078090201F0B0FCDBE7122063E7C04647
:10251000A60BFF1F6B09FF1F1A09FF1F1C09FF1FD6
:102520004809FF1F4866FF1F2309FF1F1B09FF1FE4
:102530002109FF1F2C09FF1F0010004010B50029C2
:1025400001D001F0B9FD10BDF7B5604B019199784C
:10255000A1239B004B435E4A060014681022E41836
:10256000D6235B00E0583623FF33E35C0027934318
:10257000222B41D1574B0F3A1A600760012501F019
:102580001BFE019B1880E8235B00E35C002B01D05D
:10259000B34258DD0023504FFB70AD33FF33E35897
:1025A0001A68002A03D09B88DB439B071DD0382381
:1025B000FF33E35C002B18D09B235B00E35C002B14
:1025C00013D1D133FF33E35CB3420EDAA4235B00B3
:1025D000E15AE018090A023101F0DEFD2300012270
:1025E000FE33013E01351A87FA70E8235B00E35C95
:1025F000002B2AD0A8B2FEBD03683D00002BBED040
:1026000081880430090A023101F0C6FDD6235B003F
:10261000E3581F60B2E72300B133BA00FF33985884
:10262000013781880430090A023101F0B5FDE82341
:102630005B00E35CBB42EEDCE822F61AED180023F7
:102640005200A354A6E70027F1E7200001F0CCFBDD
:1026500000281FD0002E1DDD73198826471901930D
:10266000B600200001F018FD5A30800020184068A4
:10267000013581880430090A023101F08DFD200006
:1026800001F062FCA3590133A351BD4202D0019B6A
:102690009D42E6D1114BE35C002BABD095239B0010
:1026A000E35C002BA6D00E4BE15A0029A2D00D4AC4
:1026B000A35C994202D90133A3549BE700231A215A
:1026C0002000A35401F050FB94E7C046300DFF1FDB
:1026D0003409FF1F00140340E010FF1F5A020000DE
:1026E000720200005E020000F8B51D4B1D4F1A7803
:1026F000002A10D1BA7B002A02D101321A7003E0FD
:10270000032AFAD0022AF8D001F05EFB0022012051
:10271000154B1A70F8BD154B154D1C68154B9E785E
:1027200001232B702878C0B200F0CEFCBB7B002BBD
:102730000BD101F049FCA1239B007343E4188323D0
:102740009B00E41823782B70E4E7032B02D101F0FF
:10275000F3FCF0E70020022BDCD101F055FBEAE7A7
:102760001C09FF1FA60BFF1F2309FF1F3409FF1FB2
:10277000490AFF1F300DFF1FF0B587B00EAD2F784F
:102780000FAD2D780593AC46634614000E4D0CAA90
:1027900012782E7803930D9B009201932200059BE3
:1027A000029701F029FD2E70012C01D0042C08D1D4
:1027B000802206498B889343054A1278D20113433D
:1027C0008B8007B0F0BDC0461C09FF1F6C11FF1FB6
:1027D0007809FF1F0B001B3B70B504003020E02B75
:1027E0000DD81300E025493BFF3B9BB2ED00AB4207
:1027F00005D8034B200019825A8201F045FB70BDB9
:102800008410FF1F10B501F097FA054B00205B689C
:10281000052B04D9034A5268D20200D4980810BD8F
:1028200000100040FCE100E070B501F02DFC0D4B04
:102830001B68FC33DC691D6AFFF7E4FF64198442FE
:1028400004D2094B01241B68002B07D0042200246A
:10285000064B1A70064A93690133936101F094FCA8
:10286000200070BD4866FF1F9809FF1F2309FF1F46
:10287000FC0FFF1F70B50C4D2B68FC335C6A01F038
:1028800003FCFFF7BFFF2B680025FC339B6AE318AE
:10289000834204D2054B1B68AB4200D1051B01F0FB
:1028A00073FC280070BDC0464866FF1F9809FF1FD3
:1028B000D722044B92009B5810B5002B00D09847AC
:1028C00010BDC0460000FF1FF0B587B001F08AF9C7
:1028D000FFF7EEFFC54BC64C04931B78022B45D186
:1028E000C44B1B68186A01F067FAC34BC34A1A60ED
:1028F000C34BC44A1A60A022C34B52001A60049B07
:10290000187801F019FBC149C14801F095FAC14995
:10291000C14801F091FA1022C04BFF201A608022BA
:1029200052031A60802292031A60802212041A60F5
:1029300001F052FC012001F077FCFA20400001F088
:102940009BFB582001F008FAB54801F00DFB01206F
:1029500001F0DAF9072001F0CFF9E26DB14B1A402E
:1029600084235B001343E36507B0F0BD01F004FB73
:10297000AD4E0290322001F01FFA33681B0628D4B6
:102980003C2001F019FA0F2001F016FA974B1B7842
:10299000012B00D113E1802533682B4200D0A1E048
:1029A000636C03202B43636401F006FA01F0E4FA40
:1029B000029B0299C31A5A1E814200D81A009B4BEF
:1029C0001A608C4B19681E235343994A9B18CB619C
:1029D0008BE701F0D1FA8023E26BDB021343039013
:1029E000E363E26D8F4B03201A4028231343E36512
:1029F00001F0E2F90320A56E01F0DEF9A36E0320D9
:102A0000DB03DB0B019301F0D7F9A76EED03FF03A6
:102A1000ED0BFF0B874AAB18C22B2ED8019B9B18DE
:102A2000C22B2AD8BB18C22B27D8019B2A009D4253
:102A300000D21A00019B9D4200D91D003B00974225
:102A400000D21300BD4200D93D005B1B122B14D8ED
:102A50000C2233681420934333603368764A134062
:102A6000336001F0A9F90821A36EE26DDB038A430C
:102A7000E265724ADB0B136085E7032001F09CF9E5
:102A8000A36EDB03DB0B059301F076FA039B03993E
:102A9000C21A531E814200D81300694A93421BD9BF
:102AA000FF23356864492D0A1D4032686B1C1B06E4
:102AB0000A401B0C134333600C23326800209A43F6
:102AC000083B1343336001F06FFA5E485E4BA84049
:102AD000984205DCFEF736FF019D0197059F99E7B7
:102AE0005A48F7E700235A4E33608023226CDB02FA
:102AF00013432364636C03202B43636401F05CF98C
:102B00003368013333608023626C5B021343636478
:102B100005230193E26D434B03201A404D4B1343B1
:102B2000E36501F049F90821A26EE36D434F8B4341
:102B3000E3653B6802394B43D203D20B9A420CD86F
:102B40009B1A3B2B0BD8E36D43490B40E365636C49
:102B50000B406364414B1A6028E7D31AF1E7019BED
:102B6000013BDBB20193002BD4D1E36D3A4A134011
:102B7000E365636C134063643368042B07D9BFF3C8
:102B80004F8F374B374ADA60BFF34F8FFEE7636CE6
:102B90000320AB43636401F00FF9E26D214B032086
:102BA0001A4028231343E36501F006F90822A36EB7
:102BB000DB03DB0B3B60E36D9343E3659AE707229E
:102BC000E36B1340012B02D1002001F0B5F9264D33
:102BD000264AAB6802201340AB6001F0EDF8802379
:102BE000AA685B001343AB60E0E6C0464A0AFF1FD9
:102BF00000F000404866FF1F000003400180063DD2
:102C0000BC00034034080000A4000340710200002F
:102C100014100040FFFF3F002810004000E100E0DA
:102C20003075000000FEFEFFC4F000403066FF1F5C
:102C30007206000091FCFFFFFF00FFFF3866FF1FD8
:102C4000E30C0000E88000005F361E0060361E00C6
:102C5000A444FF1F28000100FFFFFEFF3466FF1F92
:102C600000ED00E00400FA053CF00040FFFEFFFF2D
:102C7000694E336888331B6883F3088801F0D4F900
:102C800000F018FC654B664A1B68934207D0002091
:102C900001F08AF90221634A13688B431360FFF73E
:102CA00013FE614B614C1878C0B201F03DFA00236D
:102CB000A3600233A3605E4B0120236001F07CF827
:102CC0000323A36001F058F9040001F035F8050072
:102CD00001F052F9574B186001F05EF9564B196834
:102CE000621A531EA14200D213008022D2039342E3
:102CF00001D39B029B0A3268D16AC90700D478E0ED
:102D00004E491C0C09689BB24C4359432402090AE2
:102D1000641803274A49FC3293680A6849489B1A99
:102D2000494A4A4E12684A499B18414A34609A18E7
:102D30003B400193036892089C46019B0A606344F0
:102D40000360042B03D901323B400A6003600B6827
:102D50004049E418200001F06FF93F4F3D493B68BE
:102D6000C3183B602000019300F0D6FF3B4C206865
:102D7000081838492060884205D9019B01333B601F
:102D800000F0CAFF216001F00FFA354B1B78002BD1
:102D90000ED000F0D1FF3168324B4A1B1B6812186D
:102DA0009A4233D2591A4919091A2F4801F044F8A6
:102DB0002E4C237A002B0FD000F0BEFF3168E36861
:102DC0004A1B1218934224D9591A4919091A28483A
:102DD00001F032F800232372264B83F3088801F0B8
:102DE00023F8022000F0F8FF002001F0DDF801F0E8
:102DF00023FADC0199000234641A5900641A09218B
:102E00004B438033CB40A408E41882E7FA218900C1
:102E1000CBE71949DBE7C0464866FF1F0C0AFF1FD6
:102E2000B641210310000040490AFF1F1410004062
:102E3000C4090000100AFF1F340AFF1F380AFF1FD1
:102E4000200AFF1F280AFF1F1C0AFF1F2C66FF1FF6
:102E5000240AFF1F710200006008FF1F2C0AFF1FD9
:102E60001C09FF1FE408FF1F00100040740BFF1F28
:102E70003C10004000000020DC050000A022054BB3
:102E800092009B5810B5002B01D0984710BD00F060
:102E90007BFFFBE70000FF1FA122054B92009B5820
:102EA00010B5002B01D0984710BD00F06DFFFBE777
:102EB0000000FF1FA222054B92009B5810B5002B6B
:102EC00001D0984710BD00F05FFFFBE70000FF1F37
:102ED000A322054B92009B5810B5002B01D09847B8
:102EE00010BD00F051FFFBE70000FF1FA422054BBF
:102EF00092009B5810B5002B01D0984710BD00F0F0
:102F000043FFFBE70000FF1F70B500F015FF514BBA
:102F10001860042000F060FF01F0A6F80400C30769
:102F200002D401F019F970BD00224B4B1A604B4BD3
:102F30001878013804282CD800F0CAFE03231B1F80
:102F40002700200001F000F90128ECD0444C237840
:102F5000042B71D100F0D0FF002806D001F04CF80E
:102F6000582000F0F9FE02232370032000F034FF04
:102F7000D9E7200000F0B0FFE6E7200000F0A4FF52
:102F8000E2E7200001F0F8F8DEE7200000F084FF1F
:102F9000DAE701F041F80500012808D1314B1B7830
:102FA000053B012B03D82000FFF768FFCEE72C4B31
:102FB0001B78022B01D0052B20D1022D28D12A4BC2
:102FC0009B7BAB431CD12000FFF766FF254B187895
:102FD0000128BBD16405B9D4234925224B7B034288
:102FE00005D1233A13405A42534126331A000B7D30
:102FF0009342ABD9322000F05FFFA7E7022D07D143
:10300000184B1B78052B11D12000FFF753FFDDE78C
:10301000012D0BD1012B03D12000FFF759FF95E7BC
:10302000062B03D12000FFF761FF8FE7200000F09F
:10303000ABFE022D8AD1C9E7032B04D10B4B987C40
:1030400001F00AF891E7072B8FD1094B987B00F02C
:103050006BFE8AE79C09FF1F9809FF1F9009FF1F5D
:103060002309FF1F1C09FF1FA60BFF1FBC0BFF1F1F
:10307000D40BFF1FFA210A4B0A4A49001A640A4A74
:103080005A500A4A04395A50094A08319A64094A7E
:103090005A50094A5C315A50084ADA667047C046AD
:1030A0000000FF1F7927FF1F7528FF1F2928FF1F1A
:1030B0008123FF1FE926FF1F011EFF1FD51DFF1FD4
:1030C00010B500F0EDFD10BD8023F7B59C46264BF2
:1030D000264F01932649274A274D284C284B022882
:1030E0001AD1604638600868264E30408026360384
:1030F0003043086001990978002909D11660224AF5
:103100002A60224A2260E02219689143A03A1BE01B
:103110008021C9021160F2E766463E600F68194ED1
:103120003E408027FF023E430E6001990978002946
:103130000DD1176001280ED1154A2A60154A226068
:10314000E02219689143C03A0A431A60F7BD802112
:1031500089021160EEE7E0210F4A02432A600F4A1C
:1031600022601A688A43F0E74B0AFF1FE000034021
:10317000D80003409000034000000340500003408B
:1031800040000340FFFFE3FF0280063D8045082228
:103190000180063D8066082200800698805508223E
:1031A000F8B51E4B80261A680020140034403242C5
:1031B00032D11A681A4F32431A6001223B68063036
:1031C00093433B6000F0F8FD0122164D2B681E432F
:1031D0002E603B680A2613433B608027BF00124BDA
:1031E0001B683B4211D1013EF6B2FF2E09D17E226F
:1031F0000E4B1C682B68E40B1440934323432B6055
:1032000005E0082000F0D8FDE9E7002EEFD180228C
:103210002B68600893432B60F8BDC046C4F00040A3
:103220005CF0004018F0004068F0004060F00040A2
:1032300010B500F009FE01215820034A00F0ECFF10
:10324000FFF7AEFF10BDC046600AFF1F10B5782221
:103250000021034800F058FF00F096FE002010BD4A
:103260005069FF1F70B5040000F00EFF00230C2012
:103270000B4A010059438D18515C00290DD0A14221
:1032800008D1012300246B7000F046FF00F07CFFA2
:10329000200070BD01330A2BEBD11224F6E7C046A3
:1032A0005069FF1F70B5040000F0EEFE0023190006
:1032B0001D000D4A1078002806D0A0420CD1557090
:1032C00001310C320A29F5D1002B0AD100F05CFE45
:1032D00000F05AFF002070BD5078461EB0411B1808
:1032E000EEE700F019FFF3E75069FF1FF7B50400A0
:1032F0000C20002384460E4D019267465F43E85D33
:103300007E19A04212D000280BD10A4B9C4662467F
:103310001B7808331370019B70707C557160B3602B
:10332000FEBD01330A2BE8D10320F9E70720F7E7B8
:103330005069FF1F4C69FF1F8020F8B5484BC0053E
:103340001B68C1248360474BFF251A680123134380
:103350004361454BA4001A68444B40211A60444B1A
:103360001A68444B1A60444B1A59AA431A51C52291
:1033700092009E58AE433143802699509F583F4952
:10338000F6010F403E439E509E5880273602360A73
:103390003043985080201A5900020A4002431A51C3
:1033A00004341A59364E3F04324080263A431A51AB
:1033B0001A5936061202120A32431A5108341A599F
:1033C00080260A4002431A51C32292009F58B446F5
:1033D000AF4337439F509F58294E0F4007439F509C
:1033E0009F58374080263604374380269F509F5889
:1033F00036063F023F0A37439F50C0221F59AF4352
:103400003A431A511A591202120A1643C6221E5181
:1034100092009C58AC4365462C439C509C58002518
:103420000C4020439850C72080001A58154C11407A
:10343000C02212020A431A50134B1B78DB08AB421E
:1034400001DC0020F8BD2378002B06D0A368002BF8
:1034500000D0984701350C34EEE71220F2E7C04661
:103460003C45FF1F3845FF1FB0F000404869FF1F73
:10347000B4F000404469FF1F00E100E0FF00FFFFDF
:10348000FFFF00FF5069FF1F4C69FF1F030010B5CD
:103490001F2809D8072200201340072404490A786E
:1034A000A24313430B7010BD00230620F5E7C0466E
:1034B0004C69FF1F034A0449136800200B40136046
:1034C0007047C0461CF00040FFFFC1FF054B064996
:1034D0001B780A6805485B0702401B0B134300205A
:1034E0000B6070474C69FF1F1CF00040FFFFC1FFDD
:1034F00070B50C25FFF7EAFF0A4B1C780A4BE4086D
:103500006543ED18002C01D1200070BD2B78002BF5
:1035100006D06B68002B00D09847013C0C3DF1E7CA
:103520001220F2E74C69FF1F4469FF1F07B5042210
:10353000074801A900F034F9019B013305D180232C
:10354000044ADB0411680B43136000200EBDC04623
:103550001C18001114F00040F0B505002026184B8F
:1035600087B00493049B002B03D11124200007B0E3
:10357000F0BD002102220B0001910091052000F016
:10358000A3FD02230F490A681A42FCD10596059C47
:10359000631E0593002CFAD10B4A1368002BFCDA4A
:1035A0000F276F440121380000F026FC3B782B42A6
:1035B000DCD0052000F000FC049B013B0493D1E724
:1035C000FFFFFF0790C8004000C8004007B500F0AB
:1035D0005BFD80220821D205936A0191002B01D165
:1035E0000739916202210C4A11600199481E01902D
:1035F0000029FAD103311160053101910199481E6A
:1036000001900029FAD11160002B02D18022D2054D
:10361000936200F0B9FD07BD00C00040F0B52D4C2D
:1036200089B02378002B4FD1FEF76CF902232A4F83
:1036300003903A681A42FCD120230693069B5A1E37
:103640000692002BFAD1254E3368002BFCDA0120BC
:10365000FFF782FF011E02D0112009B0F0BD030068
:1036600003220190009005AD9F2000F02DFD032165
:10367000280000F0C1FB02233A681A42FCD1202343
:103680000793079B5A1E0792002BFAD13368002B31
:10369000FCDA0120FFF760FF0028DDD10398FEF778
:1036A00045F9AA786B7811041B020B4329780B4368
:1036B00063601300113B0A49052B07D8012393408F
:1036C000A3600B60012323700020C6E780231B0347
:1036D000F6E7C0462445FF1F90C8004000C80040E0
:1036E0009808FF1F1E4B30B55A6818781D4B85B0DF
:1036F000D31859424B4101210093002300F00CFCE8
:10370000194B1A4A02259A6300221A6510325A652B
:103710008022C4219D65164B1648D202DA678900C3
:103720004258154B80241A4080231B0413434350F6
:10373000642341200393E40500F078F9402000F071
:1037400075F96562039D6B1E0393002DFAD1032367
:103750006362FFF73BFFA562FFF760FF05B030BD76
:103760003045FF1F95FFFEF700C80040050001FF30
:1037700004E100E000E100E0FFFF00FF10B5064BB0
:1037800018705960FFF7AEFF00211320034AFFF7BE
:10379000ADFD002010BDC0463045FF1FE536FF1FC0
:1037A000F0B5040085B003920291FEF7ABF88822D1
:1037B00063035B0B52051A438023DB059D6A80235C
:1037C000274F0092BA68002601901B039A420CD939
:1037D000F82326001B041E401C4206D08022214BE9
:1037E00052025E6219680A431A60002D0BD100F084
:1037F0004BFC02221C4B1A608023DB055A62013A03
:103800009A6200F0C1FC0023039A934220D1002D5C
:103810000AD100F039FC144B03221D608023DB0524
:103820005A629D6200F0B0FC8023BA681B039A4282
:1038300008D9002E06D000220A4B0C495A621A6899
:103840000A401A600198FEF771F8002005B0F0BD3B
:10385000009A0299D2181278CA540133D4E7C046AC
:103860002445FF1F00C8004000C00040FFFFFEFFCE
:10387000F0B587B0029103920400FEF743F801907F
:1038800000F002FC802302250122234EDB05356077
:103890005D629A6200F078FC204F3B682B42FCD1BD
:1038A00020230493049B5A1E0492002BFAD11C4D32
:1038B0002B68002BFCDA0120FFF74EFE002802D017
:1038C000112007B0F0BD2000039A029900F064FABD
:1038D000022304003A681A42FCD120230593059B79
:1038E0005A1E0592002BFAD12B68002BFCDA01201E
:1038F000FFF732FE051EE3D100F0C6FB8023032252
:10390000DB0535605A629D6200F03EFC0198FEF7CF
:103910000DF8E0B2D5E7C04600C0004090C80040B6
:1039200000C80040F0B5802687B00400FDF7EAFF2C
:10393000F605B36A02250393029000F0A5FB01236C
:10394000244F3D607562B36200F01EFC224E336866
:103950002B42FCD120230493049B5A1E0492002B7B
:10396000FAD11E4D2B68002BFCDA0120FFF7F4FD85
:10397000002802D0112007B0F0BD200000F0B4FBF9
:103980000223019032681A42FCD120230593059B43
:103990005A1E0592002BFAD12B68002BFCDA03206B
:1039A000FFF7DAFD041EE5D100F06EFB8023032251
:1039B000DB053C605A629C6200F0E6FB039B002B37
:1039C00001D1FFF703FE0298FDF7B0FF6B461879AF
:1039D000D1E7C04600C0004090C8004000C8004089
:1039E00007B5000201910422000A01A9FFF740FF78
:1039F0000EBD000073B5050005240B4AA3005B4211
:103A00009B1819686B46DE1D300000F035FA02285D
:103A100004D133782B55013CEFD276BD052CFCD078
:103A20000128FAD10230F8E7140900111F2807D83D
:103A3000012380228340D20591680B439360704735
:103A40003F2808D80123802220388340D2055169BD
:103A50000B435361F3E75F28F1D8012380224038FC
:103A60008340D205116A0B431362E8E71F2807D889
:103A7000012280218240C9058B6893438B60704787
:103A80003F2808D80122802120388240C9054B698F
:103A900093434B61F3E75F28F1D80122802140383E
:103AA0008240C9050B6A93430B62E8E71F2810D8D0
:103AB00080230200DB05153A1968012A06D8202266
:103AC0009143196019680A431A60704701228240C5
:103AD000F6E73F2811D880230200DB05353AD96884
:103AE000032A06D810229143D960D9680A43DA60C4
:103AF000EBE7012220388240F5E75F28E5D8422332
:103B00008022181A413B8340D205516A9943516281
:103B1000516A0B435362D8E710B50400012813D152
:103B2000A022184992050B685B015B0913430B60E7
:103B3000154B164A19681140154A0A431A6040226B
:103B400019680A431A6010BD0028FCD101000A2040
:103B500000F012F921000B2000F00EF9C0220A4BF0
:103B6000920019680A4340211A601A688A431A6051
:103B7000B022044912060B685B015B0913430B601A
:103B8000E1E7C04614F000401CF000407F00FEFF5B
:103B900080FD010072B6074A1368013313600422E6
:103BA000054B1A600023054A13608022D20553603A
:103BB000FEE7C0467808FF1FC0F00040C4F0004098
:103BC000044B054A1A60054B1A600022044B1A6028
:103BD0007047C046140AFF1F841E0000380AFF1FEA
:103BE000C4F000400023034A1360034A1360034AF1
:103BF0001360704754F0004040F1004044F1004031
:103C0000002310B5184C8AB0009301932378012B40
:103C100027D06946012000F01FF9002817D1009B2A
:103C200012490293019B06AA0393114B02A81B6839
:103C30000493104B1B68059300F086F810220E4980
:103C400006A800F071F9002804D1FF23237000209A
:103C50000AB010BD0123094A074902A8237000F0E9
:103C600073F80120F4E7C0464C66FF1F10290011CD
:103C7000082900110C290011202900115066FF1F8E
:103C800013B501246946012000F0E6F8034B0094C7
:103C90000193FFF7B5FF200016BDC046BB0B000027
:103CA00010B5FFF79FFFFFF7EBFF002802D0024B94
:103CB000984710BDFEE7C046E1A2000002B471467D
:103CC00049084900095649008E4402BC7047C04665
:103CD00002B4714649084900095C49008E4402BC9F
:103CE0007047C04603B47146490840004900095A6C
:103CF00049008E4403BC704701B40248844601BCAD
:103D0000604700BFF90D010001B40248844601BCC0
:103D1000604700BFE512010001B40248844601BCBF
:103D2000604700BF090E000001B40248844601BC90
:103D3000604700BFC1F7000001B40248844601BCDF
:103D4000604700BFC95C010001B40248844601BC61
:103D5000604700BFDD3F000001B40248844601BC5B
:103D6000604700BF7912010001B40248844601BCDB
:103D7000604700BF53B9000001B40248844601BC4B
:103D8000604700BFC59E001101B40248844601BCD3
:103D9000604700BFE917010001B40248844601BC36
:103DA000604700BF9573010001B40248844601BC1E
:103DB000604700BF85C1000001B40248844601BCD1
:103DC000604700BF0189000001B40248844601BC7D
:103DD000604700BFA9D8000001B40248844601BC76
:103DE000604700BF1907010001B40248844601BCC6
:103DF000604700BF71B0000001B40248844601BCB6
:103E0000604700BF3D71010001B40248844601BC17
:103E1000604700BF19FA000001B40248844601BCA3
:103E2000604700BF8B52010001B40248844601BCC8
:103E3000604700BF7997000001B40248844601BC86
:103E4000604700BF2D6C010001B40248844601BCEC
:103E5000604700BFED68010001B40248844601BC20
:103E6000604700BFE1AC000001B40248844601BCD9
:103E7000604700BFB352010001B40248844601BC50
:103E8000604700BF9938001101B40248844601BC64
:103E9000604700BF116E000001B40248844601BCB7
:103EA000604700BFF935010001B40248844601BCF7
:103EB000604700BFC1A5000001B40248844601BCB0
:103EC000604700BF6137010001B40248844601BC6D
:103ED000604700BF0534010001B40248844601BCBC
:103EE000604700BF0934010001B40248844601BCA8
:103EF000604700BFE94C010001B40248844601BCA0
:103F0000604700BF01D7000001B40248844601BCED
:103F1000604700BFE90B010001B40248844601BCC0
:103F2000604700BFC56D010001B40248844601BC72
:103F3000604700BFCD4C010001B40248844601BC7B
:103F4000604700BFEDA5000001B40248844601BCF3
:103F5000604700BF5976010001B40248844601BCA5
:103F6000604700BF6D0B010001B40248844601BCEC
:103F7000604700BF8D11010001B40248844601BCB6
:103F8000604700BF156B010001B40248844601BCC4
:103F9000604700BFADAE000001B40248844601BCDA
:103FA000604700BFC166010001B40248844601BCFD
:103FB000604700BF016C010001B40248844601BCA7
:103FC000604700BFE927000001B40248844601BCF5
:103FD000604700BFE9F6000001B40248844601BC16
:103FE000604700BFF9A6000001B40248844601BC46
:103FF000604700BF8937010001B40248844601BC14
:10400000604700BF6DF6000001B40248844601BC61
:10401000604700BF0D52010001B40248844601BC54
:10402000604700BFDD0C010001B40248844601BCBA
:10403000604700BFC9A9000001B40248844601BC22
:10404000604700BF090E000001B40248844601BC6D
:10405000604700BF8944000001B40248844601BCA7
:10406000604700BF4DF9000001B40248844601BC1E
:10407000604700BFBD0B010001B40248844601BC8B
:10408000604700BF8512010001B40248844601BCAC
:10409000604700BF75A9000001B40248844601BC16
:1040A000604700BFD9B0000001B40248844601BC9B
:1040B000604700BFF9ED000001B40248844601BC2E
:1040C000604700BFE9D4000001B40248844601BC47
:1040D000604700BF496D010001B40248844601BC3D
:1040E000604700BFBD5C010001B40248844601BCCA
:1040F000604700BFA96F010001B40248844601BCBB
:10410000604700BFA1AF000001B40248844601BC73
:10411000604700BFB70E000001B40248844601BCEE
:10412000604700BF21A9000001B40248844601BCD9
:10413000604700BF8914010001B40248844601BCF5
:10414000604700BF75F8000001B40248844601BC16
:10415000604700BF0134010001B40248844601BC3D
:10416000604700BFDD0A010001B40248844601BC7B
:10417000604700BF51B8000001B40248844601BC4A
:10418000604700BFF535010001B40248844601BC18
:10419000604700BF9DA9000001B40248844601BCED
:1041A000604700BFC115010001B40248844601BC4C
:1041B000604700BFD544010001B40248844601BCF9
:1041C000604700BFCD0C010001B40248844601BC29
:1041D000604700BF8D82000001B40248844601BCE4
:1041E000604700BFED6B010001B40248844601BC8A
:1041F000604700BFB1B2001101B40248844601BC5F
:10420000604700BF9D6A000001B40248844601BCBB
:10421000604700BF2144000001B40248844601BC4D
:10422000604700BF0167010001B40248844601BC39
:10423000604700BF6911010001B40248844601BC17
:08424000604700BF8552010038
:1042480002000000DABB001101000000A8B900114B
:1042580002000000D6BB0011010000008842FF1FC9
:1042680002000000B0B90011010000009463FF1FB4
:1042780002000000D4BB0011030000000863FF1F08
:104288001200000002000000DABB0011010000006B
:10429800F0B9001102000000D6BB001101000000B7
:1042A800EDB9001102000000FAB900110300000086
:1042B8004363FF1F02000000D4BB0011030000008D
:1042C8005863FF1F02000000D6BB00110100000068
:1042D800ECB9001102000000F8B900110300000059
:1042E8001963FF1F02000000D4BB00110300000087
:1042F8003A63FF1F02000000DABB00110100000052
:1043080034BA001102000000D6BB00110100000001
:10431800D143FF1F0200000046BA0011010000004F
:104328002BBA001102000000D6BB001101000000EA
:10433800D043FF1F0200000044BA00110100000032
:104348006063FF1F02000000D6BB001101000000DF
:10435800CF43FF1F0200000042BA00110100000015
:104368001BBA001102000000D6BB001101000000BA
:10437800CE43FF1F0200000040BA001101000000F8
:1043880016BA001102000000D6BB0011010000009F
:10439800CD43FF1F020000003EBA001101000000DB
:1043A80011BA001102000000D6BB00110100000084
:1043B800CC43FF1F020000003CBA001101000000BE
:1043C8000CBA001102020202020200000000000002
:1043D80016150000894B00114D4B001188BA0011C9
:1043E800900118001800FFFF0701020304050602E8
:1043F80001060000000000000000000000000000AE
:1044080000000000000000000000000000000300A1
:1044180002000000DABB00110100000008BB001117
:1044280002000000D6BB0011010000008844FF1FF5
:104438000200000012BB0011010000008E63FF1F84
:1044480002000000D4BB001103000000FC65FF1F40
:1044580002000000D6BB0011010000008844FF1FC5
:104468000200000010BB0011010000009063FF1F54
:1044780002000000D4BB001103000000F465FF1F18
:10448800120000000001000000000111FFFF000001
:1044980050485936000000000000000001000000EC
:1044A80099BA00110B000500F7000000B4000028BD
:1044B800002800283075A000A000A000A000000877
:1044C8000008E001F00010001000100010001000BB
:1044D800100050005000500010001000D0070000DD
:1044E800000000000F0001000500307507001000F3
:1044F800010081FF00000000FF000000AD70001106
:10450800B56E0011456C0011FFFF0100FF000000AF
:10451800C99A0011459800115D970011000000002C
:104528000000000000000800040000003B00010833
:104538005902E00188212800FF0000000200000065
:10454800DABB001101000000A0BC0011020000004D
:10455800D6BB001101000000C145FF1F020000008A
:10456800D2BB001101000000086AFF1F0200000012
:10457800D6BB001101000000C045FF1F020000006B
:10458800D0BB001101000000BE45FF1F0200000063
:10459800D6BB001101000000BC45FF1F020000004F
:1045A800CEBB001101000000B445FF1F1800180021
:1045B8000000900102000003020200000200000057
:1045C800DABB001101000000B4BC001102000000B9
:1045D800D6BB0011010000000446FF1F02000000C6
:1045E800CCBB001100000000000000000200000029
:0E45F800D4BB001103000000286AFF1F20FF43
:040000051FFF184180
:00000001FF
